:100000000C946B010C9493010C9493010C94930148
:100010000C9493010C9493010C9493010C94930110
:100020000C9493010C9493010C9493010C94930100
:100030000C9493010C9493010C9493010C949301F0
:100040000C9495320C9493010C94F1050C942D06AC
:100050000C9493010C9493010C9493010C949301D0
:100060000C9493010C949301084AD73B3BCE016E4C
:1000700084BCBFFDC12F3D6C74319ABD56833DDAFF
:100080003D00C77F11BED9E4BB4C3E916BAAAABE0E
:10009000000000803F05A84CCDB2D44EB93836A937
:1000A000020C50B9918688083CA6AAAA2ABE000074
:1000B00000803F0664EC1B3C04BC163E3BE5B93CAB
:1000C000C93C37C29E5A3D660498083EEA69AAAA0E
:1000D0003E000000803F2020202020202020004ED5
:1000E0006F206D61762064617461210020202020E2
:1000F00020202020202020202020207C20202020A4
:1001000020202020202020202020207CC6202020ED
:10011000202020202020202020C5207C20202020DE
:1001200020202020202020202020207C2020202073
:100130002020202020202020202020004D696E69D2
:100140006D4F53442D457874726120322E347C43B8
:100150006F707465722072373236004368617220A6
:10016000446F6E650A00526561647920666F722083
:10017000466F6E740A0000407A10F35A00A0724E67
:1001800018090010A5D4E80000E87648170000E43C
:100190000B54020000CA9A3B000000E1F505000084
:1001A00080969800000040420F000000A0860100E9
:1001B0000000102700000000E803000000006400B9
:1001C000000000000A000000000001000000000024
:1001D0002C76D888DC674F0823DFC1DFAE59E1B148
:1001E000B796E5E3E453C63AE651997696E8E6C257
:1001F0008426EB898C9B62ED407C6FFCEFBC9C9F5E
:1002000040F2BAA56FA5F490055A2AF75C936B6C7F
:10021000F9676DC11BFCE0E40D47FEF520E6B50073
:10022000D0ED902E0300943577050080841E0800E1
:1002300000204E0A000000C80C333333330F986E91
:1002400012831141EF8D2114893BE65516CFFEE64E
:10025000DB18D1844B381BF77C1D901DA4BBE42414
:10026000203284725E228100C9F124ECA1E53D2791
:100270006E616E00696E66000000000024002700B9
:100280002A0000000000250028002B0000000000CC
:1002900023002600290004040404040404040202C8
:1002A00002020202030303030303010204081020F5
:1002B0004080010204081020010204081020000000
:1002C0000007000201000003040600000000000017
:1002D00000007B06B82B11241FBECFEFD8E0DEBF95
:1002E000CDBF14E0A0E0B1E0E4E4F1E702C0059086
:1002F0000D92A234B107D9F716E0A2E4B4E001C030
:100300001D92AD38B107E1F712E0C6EDD2E004C0AE
:100310002297FE010E949C38C23DD107C9F70E9476
:100320001C340C94A0380C940000283008F027E00E
:100330003327DA01990F311D87FD91600096610521
:10034000710539F432602E5F3D9330E32A95E1F771
:1003500008959F3F30F080387105610509F03C5FDA
:100360003C5F3D93913008F08068911DDF93CF93FF
:100370001F930F93FF92EF92192F987F9695E92F75
:1003800096959695E90FFF27E053FE4F992733275F
:10039000EE24FF24A701E70105900894079428F4B0
:1003A000360FE71EF81E491F511D660F771F881F65
:1003B000991F0694A1F70590079428F4E70EF81EFC
:1003C000491F561FC11D770F881F991F661F06946E
:1003D000A1F70590079428F4F80E491F561FC71F70
:1003E000D11D880F991F661F771F0694A1F70590EE
:1003F000079420F4490F561FC71FD81F990F661F77
:10040000771F881F0694A9F784911095177041F003
:10041000D695C79557954795F794E7941A95C1F7E0
:10042000E6E7F1E068941590159135916591959105
:1004300005907FE27395E118F10A430B560BC90B47
:10044000D009C0F7E10CF11E431F561FC91FD01D74
:100450007EF4703311F48A95E6CFE894015030F0C1
:10046000080F0AF40027021708F4202F2395022F03
:100470007A3328F079E37D932A95E9F710C07D93CC
:100480002A9589F606949795679537951795179449
:10049000E118F10A430B560BC90BD00998F02395CC
:1004A0007E9173957A3308F070E37C932013B8F74C
:1004B0007E9170617D9330F0839571E37D9370E35D
:1004C0002A95E1F71124EF90FF900F911F91CF91A2
:1004D000DF91992787FD90950895FA01AA27283082
:1004E00051F1203181F1E8946F936E7F6E5F7F4F01
:1004F0008F4F9F4FAF4FB1E03ED0B4E03CD0670F7D
:10050000781F891F9A1FA11D680F791F8A1F911DCF
:10051000A11D6A0F711D811D911DA11D20D009F41F
:1005200068943F912AE0269F11243019305D319361
:10053000DEF6CF010895462F4770405D4193B3E04A
:100540000FD0C9F7F6CF462F4F70405D4A3318F0F1
:10055000495D31FD4052419302D0A9F7EACFB4E0A2
:10056000A6959795879577956795BA95C9F700975A
:100570006105710508959B01AC010A2E06945795FB
:10058000479537952795BA95C9F7620F731F841F52
:10059000951FA01D0895CF93DF93BC018230910574
:1005A00010F462E070E0A0918B06B0918C06ED0132
:1005B000E0E0F0E040E050E021C0888199818617BA
:1005C000970769F48A819B81309719F0938382831E
:1005D00004C090938C0680938B06FE0134C068178C
:1005E000790738F44115510519F08417950708F477
:1005F000AC01FE018A819B819C01E9012097E9F60B
:1006000041155105A9F1CA01861B970B049708F4FF
:10061000BA01E0E0F0E02AC08D919C911197841717
:100620009507F9F46417750781F412968D919C91E2
:100630001397309719F09383828304C090938C06AC
:1006400080938B06FD0132964CC0CA01861B970B26
:10065000FD01E80FF91F6193719302978D939C93AD
:1006600040C0FD01828193819C01D9011097A1F6C0
:100670008091890690918A06892B41F48091D80255
:100680009091D90290938A06809389064091DA026C
:100690005091DB024115510541F44DB75EB7809191
:1006A000D6029091D702481B590B209189063091B0
:1006B0008A06CA01821B930B8617970780F0AB014D
:1006C0004E5F5F4F8417950750F0420F531F5093B2
:1006D0008A0640938906F9016193719302C0E0E0B4
:1006E000F0E0CF01DF91CF910895CF93DF93009792
:1006F00009F450C0EC0122971B821A82A0918B064C
:10070000B0918C06109709F140E050E0AC17BD079E
:1007100008F1BB83AA83FE0121913191E20FF31FFF
:10072000AE17BF0779F48D919C911197280F391F4F
:100730002E5F3F4F3983288312968D919C9113979A
:100740009B838A834115510571F4D0938C06C09325
:100750008B0620C012968D919C911397AD01009746
:1007600011F0DC01D3CFFA01D383C28321913191FF
:10077000E20FF31FCE17DF0769F488819981280FF4
:10078000391F2E5F3F4FFA01318320838A819B817D
:1007900093838283DF91CF910895FC01059061508E
:1007A00070400110D8F7809590958E0F9F1F089587
:1007B000FC016150704001900110D8F78095909530
:1007C0008E0F9F1F0895FC011382128288EE93E022
:1007D000A0E0B0E084839583A683B78387EF92E09F
:1007E000918380830895FC018089803419F421E08D
:1007F00030E002C020E030E0C9010895FC018189A9
:1008000090E00895FC0164874587668747870895CF
:1008100080E090E0089580E090E0089580E090E02E
:1008200008950895EF92FF921F93CF93DF93162FB1
:100830007A0186E060E00E94C8338BE696E060E0D3
:100840000E949C2B8BE696E060E00E949C2B8BE63E
:1008500096E069E00E949C2B8BE696E0612F0E9457
:100860009C2BC0E0D0E0F701EC0FFD1F10818BE660
:1008700096E06AE00E949C2B8BE696E06C2F0E942B
:100880009C2B8BE696E06BE00E949C2B8BE696E01F
:10089000612F0E949C2B2196C633D10521F78BE650
:1008A00096E068E00E949C2B8BE696E060EA0E944E
:1008B0009C2B8BE696E060EA0E949C2B85FDF9CF8D
:1008C0008BE696E060E00E949C2B8BE696E06CE065
:1008D0000E949C2B86E061E00E94C833DF91CF919B
:1008E0001F91FF90EF9008951F93CF93DF93EC013A
:1008F000162F86E060E00E94C8338BE696E060E049
:100900000E949C2B112319F0113059F404C08BE67E
:1009100096E0688904C068896C618BE696E00E9465
:100920009C2B86E061E00E94C833DF91CF911F913C
:100930000895EF92FF920F931F938EE1489F7001ED
:100940001124E60EF11C86E060E00E94C8330BE63D
:1009500016E0C80165E00E949C2BC8016F2D0E9423
:100960009C2BC80166E00E949C2BC8016E2D0E9442
:100970009C2B1F910F91FF90EF900895EF92FF92A3
:100980000F931F937C010BE616E0C80167E00E94FD
:100990009C2BC8016FEF0E949C2B86E061E00E94B7
:1009A000C833F70187858F5F87871F910F91FF906D
:1009B000EF900895EF92FF920F931F93FC01E7844D
:1009C0008EE1E89E700111248685E80EF11C86E018
:1009D00060E00E94C8330BE616E0C80164E00E94A4
:1009E0009C2BC80163E00E949C2BC80165E00E941B
:1009F0009C2BC8016F2D0E949C2BC80166E00E94B1
:100A00009C2BC8016E2D0E949C2B1F910F91FF9073
:100A1000EF9008951F93CF93DF93EC01162F6C375F
:100A200031F40E94BE04CE010E94DA040AC08BE6B3
:100A300096E067E00E949C2B8BE696E0612F0E9477
:100A40009C2B81E090E0DF91CF911F9108950F934F
:100A50001F9386E060E00E94C8330BE616E0C801F1
:100A600064E00E949C2BC80164E00E949C2B86E0FD
:100A700061E00E94C8331F910F9108951F938DE785
:100A800096E066E973E00E948232882361F081304B
:100A900011F412E009C0823011F411E005C0833076
:100AA00011F410E001C013E01092430410924204CC
:100AB00017C06091420470914304605F8BE696E03A
:100AC0000E949C2B8BE696E0612F0E949C2B8091CC
:100AD000420490914304019690934304809342040E
:100AE000809142049091430440971CF31F91089514
:100AF000CF93DF93EC0186E060E00E94C8338BE681
:100B000096E060EA0E949C2B8BE696E06FEF0E94D5
:100B10009C2B80FF05C080E4888B88E0898B13C004
:100B20008DE796E060E973E00E948232882319F431
:100B3000188A86E003C080E4888B88E0898B86E091
:100B400060E00E94C833DF91CF910895CF92DF9289
:100B5000FF920F931F936C0186E061E00E9489333E
:100B600082E060E00E94893382E061E00E94C83345
:100B7000C6010E94780586E060E00E94C8330BE65B
:100B800016E0C8016CEE0E949C2BC8016FEF0E941A
:100B90009C2BF82EC80160E00E949C2BF601608916
:100BA0006260C8010E949C2B62E370E080E090E0EC
:100BB0000E94EB32C8016CE60E949C2BFFEEFF22E4
:100BC000C8016F2D0E949C2BC6010E943E05C601E4
:100BD00061E00E9474041F910F91FF90DF90CF900D
:100BE00008951F920F920FB60F9211242F933F93E7
:100BF0004F938F939F93EF93FF934091C600209163
:100C00006C0630916D062F5F3F4F8091700690917A
:100C100071062823392380916E0690916F0628175C
:100C2000390779F080916C0690916D06E09172061B
:100C3000F0917306E80FF91F408330936D062093FF
:100C40006C06FF91EF919F918F914F913F912F9162
:100C50000F900FBE0F901F9018951F920F920FB616
:100C60000F9211242F933F938F939F93EF93FF93B2
:100C700020917606309177068091740690917506E2
:100C800028173907E9F08091760690917706E09170
:100C90007A06F0917B06E80FF91F80818093C600E9
:100CA0008091760690917706019620917806309192
:100CB000790682239323909377068093760610C05B
:100CC0002091740630917506809176069091770692
:100CD0002817390729F48091C1008F7D8093C100C6
:100CE000FF91EF919F918F913F912F910F900FBEA8
:100CF0000F901F9018958F92AF92CF92EF92FF9224
:100D00000F931F9382EC94E060E045EC50E024ECFC
:100D100030E000EC10E0F1ECEF2EF12CCC24C39489
:100D2000E8E9AE2E70E2872E0E94F22B8FED94E060
:100D30000E94E3031F910F91FF90EF90CF90AF902F
:100D40008F9008958091F1048130C1F40E94DD32CA
:100D500068517C4F8F4F9F4F6093F2047093F30460
:100D60008093F4049093F5041092F10490E0809144
:100D7000F604882309F491E09093F6040E94DD3292
:100D80002091F2043091F3044091F4045091F50461
:100D9000261737074807590718F481E08093F104B4
:100DA0000895EF92FF920F931F938091E30288239F
:100DB00061F49091660580917305891719F081E0BF
:100DC0008093740590937305C0C08091750584303D
:100DD000C9F590911A05892F8650823008F4B5C064
:100DE000809176058917A1F0909376050E94DD32F7
:100DF00060937705709378058093790590937A05D1
:100E0000909176058091E402981711F411E001C0E9
:100E100010E00E94DD3220917705309178054091F5
:100E2000790550917A05621B730B840B950B615DFC
:100E300077408040904008F47AC080911A058093F2
:100E4000E40275C0853029F480917B0590917C0582
:100E500014C0863029F480917D0590917E050DC0E7
:100E6000873029F480917F059091800506C08830F5
:100E700041F480918105909182059093680580935B
:100E80006705809183052091670530916805882367
:100E900049F544E0203B340740F4809173058823F2
:100EA00021F081E0809374054EC0C901805B9440BD
:100EB0008955924040F480917305813021F081E0A2
:100EC000809374050CC02950374008F43EC08091CF
:100ED00073058230D1F181E08093740582E08093C4
:100EE000730533C0215B344080F1E0907705F090CA
:100EF00078050091790510917A0588EE93E0A0E0DD
:100F0000B0E0E80EF91E0A1F1B1F0E94DD32E61634
:100F1000F70608071907C8F40E94DD3260937705C9
:100F2000709378058093790590937A0502C0112318
:100F300061F081E080937405809173058F5F8093E9
:100F40007305833010F0109273051F910F91FF907D
:100F5000EF900895AF92BF92CF92DF92EF92FF92FF
:100F60000F931F936091C0057091C1058091C205D8
:100F70009091C3052091FB043091FC044091FD0445
:100F80005091FE040E94F13620E030E040E752E448
:100F90000E94F1362DEC3CEC4CEC5DE30E94F13606
:100FA0007B018C0160915505709156058091570524
:100FB0009091580526E636E646E65FE30E94F13654
:100FC0009B01AC01C801B7010E94563460935505DE
:100FD0007093560580935705909358059091480655
:100FE000913061F580919405882341F580915405F5
:100FF000803120F19093940580E090E0A0E0B0E093
:101000008093A1059093A205A093A305B093A40596
:101010000E94DD3228EE33E040E050E00E945D386F
:1010200020934B0530934C0540934D0550934E054E
:1010300080914F0580939605809395058091540586
:101040008031B8F00E94DD326093490670934A0601
:1010500080934B0690934C068FEF9FEFAFEFBFEF5F
:101060008093EF029093F002A093F102B093F2020A
:101070002EC00E94DD322091490630914A064091EF
:101080004B0650914C06621B730B840B950B615100
:10109000774280409040D8F08091EF029091F0022A
:1010A000A091F102B091F2028F5F9F4FAF4FBF4FFF
:1010B00071F480919405813051F40E94DD32609387
:1010C000EF027093F0028093F1029093F202A090ED
:1010D0006905B0906A05C0906B05D0906C05C6019B
:1010E000B50120E030E040E85FE30E94E6361816E4
:1010F00094F5E090A105F090A2050091A305109150
:10110000A4050E94DD3220914D0630914E0640919B
:101110004F0650915006621B730B840B950B0E9477
:10112000BC359B01AC01C601B5010E94F13620E03F
:1011300030E04AE754E40E9423359B01AC01C8012A
:10114000B7010E9456346093A1057093A205809365
:10115000A3059093A405A0905005B0905105C090B0
:101160005205D090530560917105709172058827E2
:1011700077FD8095982F0E94BE3520E030E040E258
:1011800051E40E94F1367B018C010E94DD322091F6
:101190004D0630914E0640914F0650915006621B0D
:1011A000730B840B950B0E94BC359B01AC01C801ED
:1011B000B7010E94F13620E03AEB4BE55AE40E9479
:1011C00023359B01AC01C601B5010E9456346093E2
:1011D00050057093510580935205909353050E94DA
:1011E000DD3260934D0670934E0680934F069093C8
:1011F000500680919405813009F0B8C00E94DD321C
:1012000028EE33E040E050E00E945D3880914B05CD
:1012100090914C05A0914D05B0914E05281B390BBE
:101220004A0B5B0BCA01B9010E94BC356093DD0219
:101230007093DE028093DF029093E0026091470595
:10124000709148058091490590914A050E94BE35EC
:101250007B018C0120919D0530919E0540919F0559
:101260005091A0050E94E636181644F4E0929D05C0
:10127000F0929E0500939F051093A005E0905A05FB
:10128000F0905B0500915C0510915D05C801B70108
:1012900020915106309152064091530650915406C8
:1012A0000E94E636181644F4E0925106F092520677
:1012B0000093530610935406E0906905F0906A0578
:1012C00000916B0510916C05C801B7012091A5052F
:1012D0003091A6054091A7055091A8050E94E636D9
:1012E000181644F4E092A505F092A6050093A70510
:1012F0001093A805E0900805F090090500910A05F3
:1013000010910B05C801B7012091A9053091AA05DC
:101310004091AB055091AC050E94E636181644F496
:10132000E092A905F092AA050093AB051093AC05D5
:10133000E0901005F0901105009112051091130531
:10134000C801B701209155063091560640915706C5
:10135000509158060E94E636181644F4E09255065D
:10136000F092560600935706109358061F910F915E
:10137000FF90EF90DF90CF90BF90AF9008958DE7F2
:1013800096E06AE773E00E948232882399F586E648
:1013900096E6A6E6B0E48093F7049093F804A09351
:1013A000F904B093FA0480E090E0A0E8BFE38093F2
:1013B000FB049093FC04A093FD04B093FE0480E131
:1013C0008093FF048CE0809300058AEB80930105F5
:1013D0008AE08093DC0210920305109202058BE1F3
:1013E0008093040588EE93E09093060580930505AD
:1013F0008AE134C082E598EBAEE0B0E48093F70474
:101400009093F804A093F904B093FA0485E89BEE56
:10141000A1E5B0E48093FB049093FC04A093FD0449
:10142000B093FE0489E18093FF0486E68093000573
:101430008BEB8093010582E18093DC0280E89CE0E5
:1014400090930305809302058CE18093040580EA64
:1014500094E190930605809305058EE1809307053E
:101460000895CF93DF938DE796E06CE773E00E94D9
:10147000823280935E058DE796E06EE773E00E940E
:101480008232809359058DE796E060E873E00E9410
:10149000823280935F058DE796E06EE873E00E94EC
:1014A0008232809383058DE796E066E773E00E94C1
:1014B0008232809366058DE796E06AE873E00E94C9
:1014C0008232809375058DE796E064E873E00E94B0
:1014D0008232809393058DE796E066E873E00E9480
:1014E0008232809392058DE796E06CE873E00E946B
:1014F0008232809362058DE796E062E973E00E9494
:101500008232809360058DE796E064E973E00E9483
:10151000823280936105C0E0D0E0BE0168567C4F06
:101520008DE796E00E948232FE01E857FA4F8083F1
:10153000882321F02196C830D10579F7C857DA4FB2
:101540001982DF91CF910895BC018DE796E00E944A
:1015500082320895DF92EF92FF920F931F93CF9301
:10156000DF93D82E7B016091080570910905809169
:101570000A0590910B052091FB043091FC044091E9
:10158000FD045091FE040E94F13620E030E040EA74
:1015900050E40E9456342DEC3CEC4CE850E40E94A0
:1015A000F1360E948B358B019C01CB0101978B9703
:1015B00088F4C80169E070E00E944A38CFECD0E0BE
:1015C000C81BD90BC80169E070E00E944A38E60EDA
:1015D000F71E0CC00C3211051CF4CFECD0E006C095
:1015E00084E090E0E80EF91EC8ECD0E00FED14E0C6
:1015F0009EE0D90EC8016D2D4E2D0E94990400D099
:1016000000D000D0EDB7FEB73196ADB7BEB7129699
:101610001C930E93119780E091E093838283D5838E
:10162000C4830E94D12B8DB79EB706960FB6F8944F
:101630009EBF0FBE8DBFDF91CF911F910F91FF9085
:10164000EF90DF900895BF92CF92DF92EF92FF92DA
:101650000F931F93CF93DF93C82FD0E0CC0FDD1FE4
:10166000C257DF4F613009F069C0C090F704D090D5
:10167000F804E090F904F090FA04B090FF044DB73C
:101680005EB7465150400FB6F8945EBF0FBE4DBFD7
:101690000DB71EB70F5F1F4F8FED94E0ADB7BEB70C
:1016A00012969C938E93119783E091E0F8019383B7
:1016B00082838DE190E095838483C701B6012091F8
:1016C00010053091110540911205509113050E94AB
:1016D000F136D80116966D937D938D939C9319974F
:1016E0001A96BC921A971B961C921B971D96DC9318
:1016F000CE931C9721961F96DC93CE931E97C7011D
:10170000B6012091140530911505409116055091B0
:1017100017050E94F136F801608B718B828B938BD9
:10172000B48A158A0E94D12B4DB75EB74A5E5F4FCF
:101730000FB6F8945EBF0FBE4DBF52C08FED94E060
:101740009E012F5F3F4F623039F5ADB7BEB71C9792
:101750000FB6F894BEBF0FBEADBFEDB7FEB7319662
:1017600012969C938E93119789E191E093838283E3
:10177000D583C483378326838091180590911905FA
:101780009187808785E090E0938782870E94D12BA4
:10179000EDB7FEB73C961FC04DB75EB748505040FE
:1017A0000FB6F8945EBF0FBE4DBFEDB7FEB73196D2
:1017B000ADB7BEB712969C938E93119783E291E0DA
:1017C00093838283D583C483378326830E94D12B5E
:1017D000EDB7FEB738960FB6F894FEBF0FBEEDBF5B
:1017E000DF91CF911F910F91FF90EF90DF90CF90FD
:1017F000BF9008952F923F924F925F926F927F9287
:101800008F929F92AF92BF92CF92DF92EF92FF9210
:101810000F931F93DF93CF9300D000D000D0CDB7AC
:10182000DEB7182F662E20910C0530910D052A3554
:10183000310530F0C9018D549F4F8935910518F558
:1018400037FF02C02D543F4FC90137FF03C09095A9
:1018500081959F4F8A31910554F087E0882E912C15
:1018600009EDA02EB12CB8EF2B2E312C39C00A97E0
:1018700074F1A8E08A2E912CF0EDAF2EB12CE3EF9D
:101880002E2E312C2DC02B35310514F0235B30402A
:10189000C90137FF03C0909581959F4F8A3191050B
:1018A00054F077E0872E912C6BEEA62EB12C5BEFD7
:1018B000252E312C15C00A9754F048E0842E912C27
:1018C00032EEA32EB12C25EF222E312C09C099E047
:1018D000892E912C86ECA82EB12C0DEC202E312CCB
:1018E00060910E0570910F05882777FD8095982FE0
:1018F0000E94BE3527EA32E94BE25CEB0E94F136EA
:101900000E94C53720E030E040EA50E40E94F13602
:1019100020E030E040E951E40E94F1360E94543763
:1019200020E030E044E352E40E9456340E948B35BC
:10193000712E1EEBC12E1FEFD12E9B01442737FDC8
:101940004095542F29833A834B835C83BFED4B2E04
:10195000B4E05B2E4AEF5FEF240E351E60910C055C
:1019600070910D05882777FD8095982F0E94BE35D0
:1019700025E33AEF4EE85CE30E94F1360E94C5375A
:101980007B018C01B601882777FD8095982F0E94F6
:10199000BE359B01AC01C801B7010E94F1367B0145
:1019A0008C0169817A818B819C810E94BE359B016B
:1019B000AC01C801B7010E9456340E948B359B01CF
:1019C000CB0101978A35910508F071C062E170E0A2
:1019D0000E944A388B012F5F3F4FAEEEBFEF6A9FE8
:1019E000C0016B9F900D7A9F900D1124820F931F61
:1019F00062E070E00E944A386D837E83E62CE01A34
:101A00004E2D4C5F8FED94E0672D0E94990400D01D
:101A100000D000D0EDB7FEB73196ADB7BEB7129685
:101A20005C924E92119720E031E0338322838D81C6
:101A30009E818A0D9B1D958384830E94D12B4DB777
:101A40005EB74A5F5F4F0FB6F8945EBF0FBE4DBFE3
:101A50008D819E818815990554F1043011053CF55E
:101A600093E0E90EC201672D4E2D0E94990400D02B
:101A700000D000D0EDB7FEB73196ADB7BEB7129625
:101A80005C924E92119720E031E0338322834D81A6
:101A90005E81420D531D558344830E94D12B8DB727
:101AA0009EB706960FB6F8949EBF0FBE8DBFACE0F2
:101AB000B0E0CA0EDB1E7394BEE4CB16D10409F06D
:101AC0004DCF26960FB6F894DEBF0FBECDBFCF9197
:101AD000DF911F910F91FF90EF90DF90CF90BF901B
:101AE000AF909F908F907F906F905F904F903F90BE
:101AF0002F90089560911F05709120058091210518
:101B00009091220520E030E040EC51E40E94F13653
:101B100020E030E044EB53E40E9423350E94543728
:101B20000E948B359B012350304037FF03C09B013F
:101B30002B5E3F4FABE2B5E0F901EB5FFB4F8081DD
:101B40008C932F5F3F4F2831310514F020E030E0B7
:101B5000119685E0A633B80779F7109232050895FB
:101B60000F931F93282F462F8FED94E0622F0E9432
:101B700002048FED94E00E94DA0480911A05882314
:101B800019F428E231E03EC0813019F42DE231E051
:101B900039C0823019F422E331E034C0833019F4C3
:101BA00027E331E02FC0843019F42CE331E02AC060
:101BB000853019F421E431E025C0863019F426E49B
:101BC00031E020C0873019F42BE431E01BC08830AD
:101BD00019F420E531E016C0893019F425E531E02B
:101BE00011C08A3019F42AE531E00CC08B3019F4A9
:101BF0002FE531E007C08D3019F024E631E002C056
:101C000025E631E04DB75EB74A5050400FB6F89424
:101C10005EBF0FBE4DBFEDB7FEB731960FED14E0BE
:101C2000ADB7BEB712961C930E9311978AE691E05A
:101C3000938382838FE790E0958384833783268321
:101C400080911B0590E026E830E0AC01429FC00186
:101C5000439F900D529F900D1124918780870E9481
:101C6000D12B8DB79EB70A960FB6F8949EBF0FBEC4
:101C70008DBFC8010E94BE041F910F9108950F935C
:101C80001F93282F462F0FED14E0C801622F0E94EA
:101C90000204C8010E94DA0480911C0560E00E94E1
:101CA000230BC8010E94BE041F910F9108950F934A
:101CB0001F93282F462F0FED14E0C801622F0E94BA
:101CC0000204C8010E94DA048DB79EB70A970FB6C6
:101CD000F8949EBF0FBE8DBFEDB7FEB73196ADB77E
:101CE000BEB712961C930E9311978AE691E09383E8
:101CF000828383EC90E0958384838BE295E09783E5
:101D0000868387E890E0918780870E94D12B8DB7EA
:101D10009EB70A960FB6F8949EBF0FBE8DBFC8013E
:101D20000E94BE041F910F9108950F931F93282FB7
:101D3000462F0FED14E0C801622F0E940204C80173
:101D40000E94DA048DB79EB70A970FB6F8949EBF2B
:101D50000FBE8DBFEDB7FEB73196ADB7BEB71296C9
:101D60001C930E93119781E791E093838283809176
:101D70001F0590912005A0912105B0912205848333
:101D80009583A683B78385E090E0918780870E9442
:101D9000D12B8DB79EB70A960FB6F8949EBF0FBE93
:101DA0008DBFC8010E94BE041F910F9108950F932B
:101DB0001F93282F462F0FED14E0C801622F0E94B9
:101DC0000204C8010E94DA048DB79EB70C970FB6C3
:101DD000F8949EBF0FBE8DBFEDB7FEB73196ADB77D
:101DE000BEB712961C930E93119789E791E09383E7
:101DF00082838091370590913805A0913905B09183
:101E00003A0584839583A683B78380913B0590919F
:101E10003C05A0913D05B0913E0580879187A28742
:101E2000B3870E94D12B8DB79EB70C960FB6F8944E
:101E30009EBF0FBE8DBFC8010E94BE041F910F91AF
:101E400008950F931F93282F462F8FED94E0622F54
:101E50000E9402048FED94E00E94DA0480913F0515
:101E6000823011F42FE105C0833011F42FE001C05E
:101E70002AE28091400590914105883C910520F02F
:101E80008091F604811120E28DB79EB708970FB6B6
:101E9000F8949EBF0FBE8DBFEDB7FEB731960FED24
:101EA00014E0ADB7BEB712961C930E93119787E856
:101EB00091E09383828324831582809142058683F7
:101EC00017820E94D12B8DB79EB708960FB6F89453
:101ED0009EBF0FBE8DBFC8010E94BE041F910F910F
:101EE00008950F931F93282F462F0FED14E0C8017C
:101EF000622F0E940204C8010E94DA048DB79EB7C7
:101F00000A970FB6F8949EBF0FBE8DBFEDB7FEB710
:101F10003196ADB7BEB712961C930E9311978DE80C
:101F200091E0938382838091430590914405A09131
:101F30004505B091460584839583A683B7838DE0DC
:101F400090E0918780870E94D12B8DB79EB70A962B
:101F50000FB6F8949EBF0FBE8DBFC8010E94BE048D
:101F60001F910F9108950F931F93282F462F0FED68
:101F700014E0C801622F0E940204C8010E94DA0422
:101F80008DB79EB70A970FB6F8949EBF0FBE8DBF50
:101F9000EDB7FEB73196ADB7BEB712961C930E9350
:101FA000119785E991E09383828380910C0590914C
:101FB0000D059583848385E090E09783868386E092
:101FC00090E0918780870E94D12B8DB79EB70A96AB
:101FD0000FB6F8949EBF0FBE8DBFC8010E94BE040D
:101FE0001F910F9108950F931F93282F462F0FEDE8
:101FF00014E0C801622F0E940204C8010E94DA04A2
:102000008DB79EB70A970FB6F8949EBF0FBE8DBFCF
:10201000EDB7FEB73196ADB7BEB712961C930E93CF
:10202000119785E991E09383828380910E059091C9
:102030000F059583848385E090E09783868387E00E
:1020400090E0918780870E94D12B8DB79EB70A962A
:102050000FB6F8949EBF0FBE8DBFC8010E94BE048C
:102060001F910F910895EF92FF920F931F93282FC6
:10207000462F9FEDE92E94E0F92EC701622F0E94B2
:102080000204C7010E94DA048DB79EB70C970FB601
:10209000F8949EBF0FBE8DBF0DB71EB70F5F1F4FC9
:1020A000EDB7FEB7F282E1828DE991E0F80193830A
:1020B00082838BE090E095838483609147057091E3
:1020C00048058091490590914A050E94BE352091AE
:1020D000FB043091FC044091FD045091FE040E94E9
:1020E000F136F801668377838087918780910005B8
:1020F000828713860E94D12B8DB79EB70C960FB6A0
:10210000F8949EBF0FBE8DBFC7010E94BE041F91F1
:102110000F91FF90EF900895EF92FF920F931F930E
:10212000282F462F3FEDE32E34E0F32EC701622F18
:102130000E940204C7010E94DA040E94DD3228EEE8
:1021400033E040E050E00E945D3880914B05909173
:102150004C05A0914D05B0914E05281B390B4A0B3B
:102160005B0BCA01B9010E94BC356093DD0270931C
:10217000DE028093DF029093E0020E948B358B0198
:102180009C018DB79EB70A970FB6F8949EBF0FBEFD
:102190008DBFEDB7FEB73196ADB7BEB71296FC92C4
:1021A000EE92119787EA91E093838283C8016CE3F2
:1021B00070E00E944A38CB016CE370E00E944A381C
:1021C000958384838AE390E097838683C8016CE3D8
:1021D00070E00E944A38918780870E94D12B8DB78A
:1021E0009EB70A960FB6F8949EBF0FBE8DBFC7016B
:1021F0000E94BE041F910F91FF90EF900895CF931E
:10220000DF93282F462FCFEDD4E0CE01622F0E941E
:102210000204CE010E94DA048DE796E068E773E0DD
:102220000E948232813039F58DB79EB70A970FB67A
:10223000F8949EBF0FBE8DBFEDB7FEB73196ADB718
:10224000BEB71296DC93CE93119781EB91E0938306
:10225000828387E190E09583848380914F05868314
:10226000178285E290E0918780870E94D12B8DB7FD
:102270009EB70A962CC0ADB7BEB71C970FB6F894A0
:10228000BEBF0FBEADBFEDB7FEB731961296DC9361
:10229000CE9311978BEB91E09383828387E190E05B
:1022A000958384838091500590915105A0915205AA
:1022B000B091530586839783A087B18781E090E032
:1022C000938782870E94D12B8DB79EB70C960FB64D
:1022D000F8949EBF0FBE8DBF8FED94E00E94BE04A8
:1022E000DF91CF9108950F931F93282F462F0FED65
:1022F00014E0C801622F0E940204C8010E94DA049F
:102300008DB79EB708970FB6F8949EBF0FBE8DBFCE
:10231000EDB7FEB73196ADB7BEB712961C930E93CC
:10232000119785EC91E09383828380915405848397
:10233000158285E290E0978386830E94D12B8DB72A
:102340009EB708960FB6F8949EBF0FBE8DBFC8010A
:102350000E94BE041F910F910895BF92CF92DF9209
:10236000EF92FF920F931F93282F462F8FED94E04B
:10237000622F0E9402048FED94E00E94DA048091A3
:10238000F104813009F038C180913F05823028F492
:10239000DD24D394BB24B39402C0DD24BB2460911C
:1023A00055057091560580915705909158050E94EA
:1023B0008B35AB0177FF03C0509541955F4F8091FE
:1023C00059052AE0829FC0011124841795072CF437
:1023D000CC24C394DD24D39401C0CC2460915A054D
:1023E00070915B0580915C0590915D052091F704EB
:1023F0003091F8044091F9045091FA040E94F136AA
:102400007B018C0160915E0570E080E090E00E94AD
:10241000BC359B01AC01C801B7010E94E636181615
:1024200024F411E0DD24D39401C010E060915F0535
:1024300070E080E090E00E94BC3520E030E040E2B7
:1024400051E40E9423359B01AC01609143057091DA
:10245000440580914505909146050E941C3587FDF5
:102460000AC09091600580914F05891710F4992357
:1024700011F440E003C041E0DD24D3942091E10257
:102480003091E2028091610590E0281739075CF4F1
:102490002D593F4F41F080916205882321F431E0AE
:1024A000DD24D39401C030E0809163058823C9F412
:1024B000DD2069F08B2D90E001968C0D911D810F30
:1024C000911D840F911D830F911D029739F48DEC9E
:1024D00091E0909365058093640503C081E080934B
:1024E000630580916305813069F491E0B91639F490
:1024F0008AED91E0909365058093640503C082E0C6
:102500008093630580916305823069F4A1E0CA1667
:1025100039F487EE91E0909365058093640503C0DC
:1025200083E08093630580916305833061F411300B
:1025300039F484EF91E0909365058093640503C0BE
:1025400084E08093630580916305843061F44130B9
:1025500039F481E092E0909365058093640503C0AF
:1025600085E08093630520916305253041F4313087
:1025700031F48EE092E090936505809364052F5FBF
:1025800020936305B1E0DB1639F480916605833052
:1025900018F41092E3020AC08091670590916805D3
:1025A000805B944018F481E08093E302263010F0C1
:1025B0001092630500D000D000D0EDB7FEB7319681
:1025C0008FED94E0ADB7BEB712969C938E931197A2
:1025D0008BE192E0938382838091640590916505FD
:1025E000958384830E94D12B8DB79EB706960FB634
:1025F000F8949EBF0FBE8DBF8FED94E00E94BE0485
:102600001F910F91FF90EF90DF90CF90BF900895B2
:10261000EF92FF920F931F93CF93DF93282F462FB4
:10262000CFEDD4E0CE01622F0E940204CE010E94C1
:10263000DA048DE796E062E773E00E948232882335
:10264000F1F000D000D000D0EDB7FEB73196ADB7B5
:10265000BEB71296DC93CE93119780E091E09383FE
:10266000828383E190E0958384830E94D12BEDB730
:10267000FEB736960FB6F894FEBF0FBEEDBF8DB70E
:102680009EB70A970FB6F8949EBF0FBE8DBF0DB7C9
:102690001EB70F5F1F4F4FEDE42E44E0F42EADB791
:1026A000BEB71296FC92EE9211978EE192E0F8017D
:1026B0009383828360915A0570915B0580915C05DC
:1026C00090915D052091F7043091F8044091F90450
:1026D0005091FA040E94F136D80114966D937D93BF
:1026E0008D939C9317978091FF0418968C9318975D
:1026F00019961C920E94D12BEDB7FEB73A960FB6F1
:10270000F894FEBF0FBEEDBFC7010E94BE04DF916B
:10271000CF911F910F91FF90EF900895EF92FF924C
:102720000F931F93CF93DF93282F462FCFEDD4E045
:10273000CE01622F0E940204CE010E94DA048DE7CE
:1027400096E060E773E00E9482328823F1F000D0C7
:1027500000D000D0EDB7FEB73196ADB7BEB7129638
:10276000DC93CE93119780E091E09383828384E1A0
:1027700090E0958384830E94D12BEDB7FEB7369607
:102780000FB6F894FEBF0FBEEDBF8DB79EB70A9788
:102790000FB6F8949EBF0FBE8DBF0DB71EB70F5F6B
:1027A0001F4F5FEDE52E54E0F52EADB7BEB7129684
:1027B000FC92EE9211978EE192E0F801938382836E
:1027C0006091690570916A0580916B0590916C0527
:1027D0002091F7043091F8044091F9045091FA04E3
:1027E0000E94F136D80114966D937D938D939C933E
:1027F00017978091FF0418968C93189719961C923E
:102800000E94D12BEDB7FEB73A960FB6F894FEBFF3
:102810000FBEEDBFC7010E94BE04DF91CF911F9193
:102820000F91FF90EF900895EF92FF920F931F93F7
:10283000CF93DF93282F462FCFEDD4E0CE01622F28
:102840000E940204CE010E94DA048DE796E06EE653
:1028500073E00E9482328823F1F000D000D000D0D3
:10286000EDB7FEB73196ADB7BEB71296DC93CE93F7
:10287000119780E091E09383828382E190E09583D9
:1028800084830E94D12BEDB7FEB736960FB6F8942D
:10289000FEBF0FBEEDBF8DB79EB70A970FB6F89477
:1028A0009EBF0FBE8DBF0DB71EB70F5F1F4F6FEDE1
:1028B000E62E64E0F62EADB7BEB71296FC92EE920D
:1028C000119786E292E0F801938382836091080574
:1028D0007091090580910A0590910B052091FB04E8
:1028E0003091FC044091FD045091FE040E94F136A9
:1028F000D80114966D937D938D939C931797809137
:10290000000518968C93189719961C920E94D12B4B
:10291000EDB7FEB73A960FB6F894FEBF0FBEEDBF07
:10292000C7010E94BE04DF91CF911F910F91FF90CC
:10293000EF900895EF92FF920F931F93282F462F49
:102940007FEDE72E74E0F72EC701622F0E9402048C
:10295000C7010E94DA048DB79EB70E970FB6F894A0
:102960009EBF0FBE8DBF0DB71EB70F5F1F4FEDB7D8
:10297000FEB7F282E1828EE292E0F80193838283D5
:1029800085E190E0958384836091550570915605AB
:10299000809157059091580520E030E040E251E4E5
:1029A0000E9423350E948B35882777FD8095982FCC
:1029B0000E94BE3520E030E040E251E40E94F13652
:1029C000F8016683778380879187809107058287E6
:1029D000138680E290E0958784870E94D12B8DB783
:1029E0009EB70E960FB6F8949EBF0FBE8DBFC7015F
:1029F0000E94BE041F910F91FF90EF900895EF92F7
:102A0000FF920F931F93CF93DF93282F462FCFED85
:102A1000D4E0CE01622F0E940204CE010E94DA04AB
:102A20008DE796E06CE673E00E9482328823F1F035
:102A300000D000D000D0EDB7FEB73196ADB7BEB72D
:102A40001296DC93CE93119780E091E0938382837A
:102A500081E190E0958384830E94D12BEDB7FEB78E
:102A600036960FB6F894FEBF0FBEEDBF8DB79EB77A
:102A70000A970FB6F8949EBF0FBE8DBF0DB71EB755
:102A80000F5F1F4FEFEDEE2EE4E0FE2EADB7BEB7A9
:102A90001296FC92EE92119786E292E0F8019383EF
:102AA000828360916D0570916E0580916F059091A4
:102AB00070050E94BE352091FB043091FC044091CA
:102AC000FD045091FE040E94F136D80114966D93D6
:102AD0007D938D939C9317978091000518968C9306
:102AE000189719961C920E94D12BEDB7FEB73A9613
:102AF0000FB6F894FEBF0FBEEDBFC7010E94BE0423
:102B0000DF91CF911F910F91FF90EF900895EF9279
:102B1000FF920F931F93282F462FFFEDEF2EF4E027
:102B2000FF2EC701622F0E940204C7010E94DA042F
:102B30008DB79EB70A970FB6F8949EBF0FBE8DBF94
:102B40000DB71EB70F5F1F4FEDB7FEB7F282E182E0
:102B50008DE891E0F8019383828360917105709113
:102B60007205882777FD8095982F0E94BE352AE050
:102B700037ED43E25CE30E94F136F801648375832C
:102B8000868397838EE090E0918780870E94D12B87
:102B90008DB79EB70A960FB6F8949EBF0FBE8DBF35
:102BA000C7010E94BE041F910F91FF90EF900895FE
:102BB000CF93DF93282F462FCFEDD4E0CE01622FA5
:102BC0000E940204CE010E94DA040E94DD3228EE47
:102BD00033E040E050E00E945D38CA01B9012CE3C7
:102BE00030E040E050E00E945D382BE132E062309E
:102BF00071058105910588F400D000D000D0EDB7B3
:102C0000FEB73196ADB7BEB71296DC93CE9311974F
:102C10003383228388E895E010C000D000D000D034
:102C2000EDB7FEB73196ADB7BEB71296DC93CE9333
:102C300011973383228385EE92E0958384830E94EB
:102C4000D12B8DB79EB706960FB6F8949EBF0FBED8
:102C50008DBF8FED94E00E94BE04DF91CF91089567
:102C6000CF92DF92EF92FF920F931F93282F462F60
:102C70008FED94E0622F0E9402048FED94E00E9499
:102C8000DA0480916205882379F40091920510E0BE
:102C90006091910570E0601B710B882777FD80952E
:102CA000982F0E94BE351CC0813039F48091910567
:102CB0008093E1021092E2023DC0883089F50091D4
:102CC000920580918105909182056AE070E00E94F2
:102CD000363810E0601B710B80E090E00E94BC353C
:102CE0006B017C016091930570E0601B710B88277C
:102CF00077FD8095982F0E94BE359B01AC01C701DE
:102D0000B6010E94233520E030E048EC52E40E94F6
:102D1000F1360E948B357093E2026093E1020AC0A3
:102D2000893041F480918105909182059093E2026F
:102D30008093E1028DB79EB70A970FB6F8949EBFB5
:102D40000FBE8DBFEDB7FEB731960FED14E0ADB7F6
:102D5000BEB712961C930E9311978AE392E0938369
:102D6000828389E090E0958384838091E102909151
:102D7000E2029783868385E290E0918780870E94B4
:102D8000D12B8DB79EB70A960FB6F8949EBF0FBE93
:102D90008DBFC8010E94BE041F910F91FF90EF905C
:102DA000DF90CF9008950F931F93282F462F8FED1C
:102DB00094E0622F0E9402048FED94E00E94DA04F6
:102DC00080919405882309F48DC000914F05202F30
:102DD00030E080919505992787FD90952817390750
:102DE000C9F10E94DD3210914F0528EE33E040E03A
:102DF00050E00E945D38CA01B90120914B05309125
:102E00004C0540914D0550914E05621B730B840B90
:102E1000950B202F30E040E050E00E9417382091C1
:102E20009605332727FD3095211B3109442737FDAF
:102E30004095542F0E945D38CA01B9010E94BC35EB
:102E400060939705709398058093990590939A05E0
:102E5000109395056091970570919805809199055B
:102E600090919A050E948B358B019C018DB79EB77E
:102E70000C970FB6F8949EBF0FBE8DBFEDB7FEB78F
:102E800031968FED94E0ADB7BEB712969C938E93BA
:102E9000119782E492E09383828387E190E09583A7
:102EA0008483C8016CE370E00E944A38CB016CE374
:102EB00070E00E944A38978386838AE390E0918786
:102EC0008087C8016CE370E00E944A38938782874C
:102ED0000E94D12B8DB79EB70C960FB6F8949EBF6B
:102EE0000FBE8DBF8FED94E00E94BE041F910F9125
:102EF0000895EF92FF920F931F93282F462FAFED67
:102F0000EA2EA4E0FA2EC701622F0E940204C70134
:102F10000E94DA048DB79EB70A970FB6F8949EBF49
:102F20000FBE8DBF0DB71EB70F5F1F4FEDB7FEB7BA
:102F3000F282E1828EE492E0F80193838283209111
:102F4000DC0230E080919B0590919C056AE070E086
:102F50000E943638CB01289FB001299F700D389F01
:102F6000700D11242091020530910305620F731F2B
:102F700080E090E00E94BC3520E030E048EC52E474
:102F80000E942335F801648375838683978380913B
:102F90000105808711860E94D12B8DB79EB70A96B6
:102FA0000FB6F8949EBF0FBE8DBFC7010E94BE042E
:102FB0001F910F91FF90EF9008955F926F927F9213
:102FC0008F929F92AF92BF92CF92DF92EF92FF9239
:102FD0000F931F93BFED6B2EB4E07B2EC3016BE00C
:102FE00044E00E940204C3010E94DA046091DD0201
:102FF0007091DE028091DF029091E0020E948B3599
:103000006B017C018090FB049090FC04A090FD0477
:10301000B090FE04509000058DB79EB7C0970FB6D4
:10302000F8949EBF0FBE8DBF0DB71EB70F5F1F4F29
:10303000EDB7FEB77282618286E592E0F801938374
:10304000828388E090E095838483C6016CE370E01E
:103050000E944A38CB016CE370E00E944A389783A3
:1030600086838AE390E091878087C6016CE370E0F5
:103070000E944A38938782878BE090E09587848707
:10308000C501B40120919D0530919E0540919F0599
:103090005091A0050E94F1360E948B35F801778788
:1030A0006687508A118A8FE890E0938B828BC501E6
:1030B000B4012091A1053091A2054091A305509142
:1030C000A4050E94F1360E948B35F801758B648B44
:1030D000568A178A84E190E0918F808F6091A505D0
:1030E0007091A6058091A7059091A8052091F704FD
:1030F0003091F8044091F9045091FA040E94F1369D
:103100000E948B35F801738F628F8091FF04848F4A
:10311000158E82E190E0978F868FC501B4012091D2
:10312000A9053091AA054091AB055091AC050E94CC
:10313000F1360E948B35F80171A360A352A213A24D
:1031400083E090E095A384A38091370590913805A2
:10315000A0913905B0913A0586A397A3A0A7B1A77E
:1031600084E090E093A782A780913B0590913C0575
:10317000A0913D05B0913E0584A795A7A6A7B7A746
:103180000E94D12B8DB79EB7C0960FB6F8949EBF04
:103190000FBE8DBFC3010E94BE041F910F91FF900F
:1031A000EF90DF90CF90BF90AF909F908F907F90E7
:1031B0006F905F900895CF92DF92EF92FF920F93FE
:1031C0001F93CF93DF93282F462FCFEDD4E0CE016E
:1031D000622F0E940204CE010E94DA046091A105D0
:1031E0007091A2058091A3059091A4052091FB0404
:1031F0003091FC044091FD045091FE040E94F13690
:103200006B017C0120E03CE34CE156E40E94E63691
:103210001816C4F58DB79EB70C970FB6F8949EBFDD
:103220000FBE8DBF0DB71EB70F5F1F4FADB7BEB737
:103230001296DC93CE93119784E992E0F801938380
:1032400082838FE890E09583848360910505709177
:10325000060580E090E00E94BC359B01AC01C701EF
:10326000B6010E942335D80116966D937D938D93F8
:103270009C931997809104051A968C931A971B9624
:103280001C9221C08DB79EB70C970FB6F8949EBFC5
:103290000FBE8DBFEDB7FEB73196ADB7BEB7129674
:1032A000DC93CE9311978DE991E0938382838FE82D
:1032B00090E095838483C682D782E086F1868091F0
:1032C0000005828713860E94D12BEDB7FEB73C968E
:1032D0000FB6F894FEBF0FBEEDBF8FED94E00E94D5
:1032E000BE04DF91CF911F910F91FF90EF90DF907F
:1032F000CF900895EF92FF920F931F93282F462FA0
:103300008FED94E0622F0E9402048FED94E00E9402
:10331000DA048091AD059091AE0564E670E00E94FC
:10332000363880E090E00E94BC3520911F05309136
:10333000200540912105509122050E9455347B01C2
:103340008C0120E030E044EB53E40E94233520E080
:1033500030E040E851E40E94F13620E030E040E8FF
:103360005FE30E9456340E9454370E948B35862FAB
:103370006093AF0567FF03C0805F8093AF058091C6
:10338000AF05882319F480E18093AF058091AF05E4
:10339000813119F481E08093AF05C801B70120E0C5
:1033A00030E044E353E40E94E63618164CF4C801BA
:1033B000B70120E030E044EB53E40E94553415C0DF
:1033C000C801B70120E030E044E353EC0E941C3513
:1033D00088234CF4C801B70120E030E044EB53E40B
:1033E0000E94563402C0C801B7010E949035709304
:1033F0001905609318058091AF0562E00E94230BC8
:103400008FED94E00E94BE041F910F91FF90EF900A
:103410000895EF92FF920F931F93CF93DF93282F7E
:10342000462F8FED94E0622F0E9402048FED94E00E
:103430000E94DA0460911D0570911E05882777FDB2
:103440008095982F0E94BE3520911F053091200550
:1034500040912105509122050E94553420E030E032
:1034600044EB53E40E94233520E030E040E851E48F
:103470000E94F1360E9454370E948B35DC01CB014B
:10348000409660E170E00E944A388F5F8093230588
:10349000E0902405F0902505009126051091270560
:1034A000C801B70120E030EC49E754E40E94E63659
:1034B00018162CF480E090ECA9E7B4E40EC0C80123
:1034C000B70120E030EC49E754EC0E941C3588231A
:1034D00064F480E090ECA9E7B4EC80932405909329
:1034E0002505A0932605B09327058DB79EB7429773
:1034F0000FB6F8949EBF0FBE8DBF0DB71EB70F5FFE
:103500001F4FCFEDD4E0EDB7FEB7D283C1838EE974
:1035100092E0F8019383828387E590E0958384832A
:1035200080E790E0978386838091280580871186C5
:10353000138612866091290570912A0580E090E03B
:103540000E94BC352091FB043091FC044091FD04A5
:103550005091FE040E94F136F801648775878687D2
:10356000978780910005808B118A0E94D12B8DB79F
:103570009EB742960FB6F8949EBF0FBE8DBF809146
:10358000230560E00E94230B80911A058A3009F020
:1035900045C0EDB7FEB770970FB6F894FEBF0FBEEB
:1035A000EDBF0DB71EB70F5F1F4FD283C18380EBF6
:1035B00092E0F8019383828380E290E09583848394
:1035C00088E590E09783868385E690E09187808701
:1035D000609124057091250580912605909127051D
:1035E0002091FB043091FC044091FD045091FE04B5
:1035F0000E94F136F80162877387848795878091EE
:103600000005868717860E94D12B8DB79EB74096FE
:103610000FB6F8949EBF0FBE8DBF10C000D000D073
:10362000EDB7FEB7D283C18386ED90E094838383A8
:103630000E94C02B0F900F900F900F908FED94E091
:103640000E94BE04DF91CF911F910F91FF90EF90E8
:1036500008950F931F93282F462F0FED14E0C801F4
:10366000622F0E940204C8010E94DA0400D000D038
:10367000EDB7FEB7128301838FED90E094838383CF
:103680000E94C02B0F900F900F900F90C8010E94C6
:10369000BE041F910F910895CF92DF92EF92FF9297
:1036A0000F931F937C01D62EC72E0FED14E0C80197
:1036B0006E2D4D2D0E940204C8010E94DA0400D034
:1036C00000D0EDB7FEB7128301838CEE90E09483B7
:1036D00083830E94C02B0F900F900F900F90C80112
:1036E0000E94BE04C70101966D2D7C2D0E94FA0B2D
:1036F000C7016D2D7C2D0E94AA0A1F910F91FF908A
:10370000EF90DF90CF9008950F931F930FED14E08B
:10371000C80165E045E00E940204C8010E94DA0485
:1037200000D000D0EDB7FEB7128301838CE391E0A7
:10373000948383830E94C02B0F900F900F900F9063
:10374000C8010E94BE041F910F9108950E94841B1E
:103750000E94BF090895EF92FF920F931F930E945A
:10376000DD320E94BC357B018C016091B005709107
:10377000B1058091B2059091B30520E030E849E0B1
:1037800055E40E9456349B01AC01C801B7010E9468
:10379000E636181694F48091EE02823039F08FEDFF
:1037A00094E00E94270582E08093EE0285E090E09D
:1037B0006AE070E00E94291B7DC28091EF02909127
:1037C000F002A091F102B091F2028F5F9F4FAF4FD4
:1037D000BF4F09F48DC20E94DD322091EF0230917B
:1037E000F0024091F1025091F202621B730B840BC4
:1037F000950B20E137E240E050E00E945D3820FD6B
:1038000077C28091EE02813039F08FED94E00E9412
:10381000270581E08093EE020E94DD174BC2609184
:10382000A4048091A20490E070E00E94AD11809108
:103830007505843010F00E94D106809174058823AC
:1038400021F48091EE02882341F08FED94E00E94F4
:103850002705109274051092EE0280917305823054
:1038600009F428C2A82FB0E0FD01EC5BFB4F80817A
:1038700081FF0BC0FD01E05BFB4F6081A25BBB4F92
:103880008C9190E070E00E94F30F80917305A82F57
:10389000B0E0FD01EC5BFB4F808182FF0BC0FD01BE
:1038A000EC5AFB4F6081AE5ABB4F8C9190E070E0B8
:1038B0000E94B30F80917305A82FB0E0FD01EC5B6F
:1038C000FB4F808183FF0BC0FD01E85AFB4F6081F5
:1038D000AA5ABB4F8C9190E070E00E94710F8091CA
:1038E0007305A82FB0E0FD01EC5BFB4F808185FFE5
:1038F0000BC0FD01E45AFB4F6081A65ABB4F8C916F
:1039000090E070E00E94210F80917305A82FB0E035
:10391000FD01EC5BFB4F808187FF0BC0FD01EC5983
:10392000FB4F6081AE59BB4F8C9190E070E00E94DC
:10393000D70E80917305A82FB0E0FD01EC5BFB4F23
:10394000808184FF0BC0FD01E859FB4F6081AA59BB
:10395000BB4F8C9190E070E00E94FF108091730546
:10396000A82FB0E0FD01EC5BFB4F808186FF0BC010
:10397000FD01E05AFB4F6081A25ABB4F8C9190E051
:1039800070E00E947A1980917305A82FB0E0FD01C4
:10399000EA5BFB4F808180FF0BC0FD01E459FB4FC8
:1039A0006081A659BB4F8C9190E070E00E94570E49
:1039B00080917305A82FB0E0FD01EA5BFB4F808189
:1039C00081FF0BC0FD01E059FB4F6081A259BB4F45
:1039D0008C9190E070E00E94950E8091B40581304A
:1039E00051F580917305A82FB0E0FD01EA5BFB4F14
:1039F000808184FF0BC0FD01E858FB4F6081AA580D
:103A0000BB4F8C9190E070E00E9433108091730561
:103A1000A82FB0E0FD01EA5BFB4F808183FF0BC064
:103A2000FD01EC58FB4F6081AE58BB4F8C9190E08C
:103A300070E00E943F0E80917305A82FB0E0FD0159
:103A4000EA5BFB4F808187FF0BC0FD01E058FB4F15
:103A50006081A258BB4F8C9190E070E00E948C1066
:103A6000809128058823A9F080917305A82FB0E0E4
:103A7000FD01EA5BFB4F808186FF0BC0FD01E4582E
:103A8000FB4F6081A658BB4F8C9190E070E00E9484
:103A9000091A80917305A82FB0E0FD01E85BFB4F88
:103AA000808182FF0BC0FD01E857FB4F6081AA5760
:103AB000BB4F8C9190E070E00E94FF1480917305E1
:103AC000A82FB0E0FD01E85BFB4F808187FF0BC0B2
:103AD000FD01E457FB4F6081A657BB4F8C9190E0EE
:103AE00070E00E94141480917305A82FB0E0FD01CE
:103AF000E85BFB4F808183FF0BC0FD01E057FB4F6C
:103B00006081A257BB4F8C9190E070E00E948E13B1
:103B100080917305A82FB0E0FD01E85BFB4F808129
:103B200081FF0BC0FD01EC56FB4F6081AE56BB4FD1
:103B30008C9190E070E00E94081380917305A82F8B
:103B4000B0E0FD01E85BFB4F808184FF0BC0FD010D
:103B5000E856FB4F6081AA56BB4F8C9190E070E015
:103B60000E94731180917305A82FB0E0FD01E85BFE
:103B7000FB4F808185FF0BC0FD01E456FB4F608148
:103B8000A656BB4F8C9190E070E00E94B00D8091E2
:103B90007305A82FB0E0FD01E85BFB4F808186FF35
:103BA0000BC0FD01E056FB4F6081A256BB4F8C91CC
:103BB00090E070E00E944C1B80917305A82FB0E04C
:103BC000FD01E85BFB4F808180FF0BC0FD01EC57DE
:103BD000FB4F6081AE57BB4F8C9190E070E00E942C
:103BE000871580917305A82FB0E0FD01E65BFB4FC0
:103BF000808183FF0BC0FD01E455FB4F6081A6551A
:103C0000BB4F8C9190E070E00E949A1480917305F4
:103C1000A82FB0E0FD01E65BFB4F808186FF0BC063
:103C2000FD01E055FB4F6081A255BB4F8C9190E0A8
:103C300070E00E94301680917305A82FB0E0FD015E
:103C4000E65BFB4F808187FF0BC0FD01EC54FB4F0F
:103C50006081AE54BB4F8C9190E070E00E94D3160F
:103C600080917305A82FB0E0FD01E45BFB4F8081DC
:103C700081FF0BC0FD01E454FB4F6081A654BB4F94
:103C80008C9190E070E00E94791780917305A82FC5
:103C9000B0E0FD01E45BFB4F808182FF0BC0FD01C2
:103CA000E054FB4F6081A254BB4F8C9190E070E0D8
:103CB0000E94DB1880917305A82FB0E0FD01E17030
:103CC000F070E65BFB4F808185FF0BC0FD01E8547F
:103CD000FB4F6081AA54BB4F8C9190E070E00E9432
:103CE000D8150E94A2061F910F91FF90EF900895A2
:103CF00080914A0480FF9BCD92CDCF93DF93EC015E
:103D00008FED94E00E94FE03C817D9073CF08FEDB9
:103D100094E00E94F303892B09F42397CE01DF91ED
:103D2000CF910895EF92FF920F931F93CF93DF935C
:103D30000091730510E08AEF90E0089F7001099FE1
:103D4000F00C189FF00C1124C70188569F4F0E9459
:103D5000A40AF801EC5BFB4F882319F08081806195
:103D600002C080818F7E808380917305C82FD0E050
:103D7000C70186569F4F0E94A40ACA59DB4F888309
:103D800080917305C82FD0E0C70184569F4F0E94D1
:103D9000A40A90E00E947D1EC859DB4F88830091E1
:103DA000730510E0C70106960E94A40AF801EC5BB7
:103DB000FB4F882319F08081826002C080818D7F53
:103DC000808380917305C82FD0E0C70108960E94B8
:103DD000A40AC25BDB4F888380917305C82FD0E0B3
:103DE000C7010A960E94A40A90E00E947D1EC05B53
:103DF000DB4F88830091730510E0C7010C960E9489
:103E0000A40AF801EC5BFB4F882319F080818460E1
:103E100002C080818B7F808380917305C82FD0E0A2
:103E2000C7010E960E94A40ACE5ADB4F8883809168
:103E30007305C82FD0E0C70140960E94A40A90E005
:103E40000E947D1ECC5ADB4F88830091730510E0E1
:103E5000C70142960E94A40AF801EC5BFB4F88233D
:103E600019F08081886002C08081877F8083809183
:103E70007305C82FD0E0C70144960E94A40ACA5A0D
:103E8000DB4F888380917305C82FD0E0C701469629
:103E90000E94A40A90E00E947D1EC85ADB4F8883CE
:103EA0000091730510E0C7014E960E94A40AF80124
:103EB000EC5BFB4F882319F08081806202C0808117
:103EC0008F7D808380917305C82FD0E0C7018096D5
:103ED0000E94A40AC65ADB4F888380917305C82FBD
:103EE000D0E0C70182960E94A40A90E00E947D1E45
:103EF000C45ADB4F88830091730510E0C701849694
:103F00000E94A40AF801EC5BFB4F882319F0808122
:103F1000806402C080818F7B808380917305C82F6D
:103F2000D0E0C70186960E94A40AC25ADB4F88835C
:103F300080917305C82FD0E0C70188960E94A40A1B
:103F400090E00E947D1EC05ADB4F8883009173056C
:103F500010E0C7018A960E94A40AF801EC5BFB4FAF
:103F6000882319F08081806802C080818F778083E8
:103F700080917305C82FD0E0C7018C960E94A40AD7
:103F8000CE59DB4F888380917305C82FD0E0C701DD
:103F90008E960E94A40A90E00E947D1ECC59DB4FB1
:103FA00088830091730510E0C701C0960E94A40A9F
:103FB000F801EA5BFB4F882319F08081816002C021
:103FC00080818E7F808380917305C82FD0E0C701E8
:103FD000C2960E94A40AC659DB4F8883809173055C
:103FE000C82FD0E0C701C4960E94A40A90E00E94A6
:103FF0007D1EC459DB4F88830091730510E0C70113
:10400000C6960E94A40AF801EA5BFB4F882319F0C8
:104010008081826002C080818D7F80838091730562
:10402000C82FD0E0C701C8960E94A40AC259DB4F2E
:10403000888380917305C82FD0E0C701CA960E947B
:10404000A40A90E00E947D1EC059DB4F8883009136
:10405000730510E0C701885B9F4F0E94A40AF80116
:10406000EA5BFB4F882319F08081806102C0808168
:104070008F7E808380917305C82FD0E0C701865B57
:104080009F4F0E94A40ACA58DB4F88838091730512
:10409000C82FD0E0C701845B9F4F0E94A40A90E024
:1040A0000E947D1EC858DB4F88830091730510E085
:1040B000C7018E5B9F4F0E94A40AF801EA5BFB4F89
:1040C000882319F08081886002C08081877F808387
:1040D00080917305C82FD0E0C7018C5B9F4F0E9471
:1040E000A40ACE58DB4F888380917305C82FD0E097
:1040F000C7018A5B9F4F0E94A40A90E00E947D1E28
:10410000CC58DB4F88830091730510E0C7018A5AB1
:104110009F4F0E94A40AF801EA5BFB4F882319F025
:104120008081806402C080818F7B80838091730551
:10413000C82FD0E0C701885A9F4F0E94A40AC658D2
:10414000DB4F888380917305C82FD0E0C701865A62
:104150009F4F0E94A40A90E00E947D1EC458DB4F2E
:1041600088830091730510E0C70182569F4F0E941B
:10417000A40AF801EA5BFB4F882319F0808180686C
:1041800002C080818F77808380917305C82FD0E033
:10419000C70180569F4F0E94A40AC258DB4F8883F4
:1041A00080917305C82FD0E0C7018E559F4F0E94A4
:1041B000A40A90E00E947D1EC058DB4F88830091C6
:1041C000730510E0C7018E599F4F0E94A40AF801A1
:1041D000E85BFB4F882319F08081816002C08081F9
:1041E0008E7F808380917305C82FD0E0C7018C59E2
:1041F0009F4F0E94A40ACE57DB4F8883809173059E
:10420000C82FD0E0C7018A599F4F0E94A40A90E0AE
:104210000E947D1ECC57DB4F88830091730510E010
:10422000C70182599F4F0E94A40AF801E85BFB4F27
:10423000882319F08081846002C080818B7F808315
:1042400080917305C82FD0E0C70180599F4F0E940D
:10425000A40ACA57DB4F888380917305C82FD0E02A
:10426000C7018E589F4F0E94A40A90E00E947D1EB5
:10427000C857DB4F88830091730510E0C70184574E
:104280009F4F0E94A40AF801E85BFB4F882319F0B6
:104290008081806802C080818F77808380917305E0
:1042A000C82FD0E0C70182579F4F0E94A40AC6576B
:1042B000DB4F888380917305C82FD0E0C7018057FA
:1042C0009F4F0E94A40A90E00E947D1EC457DB4FBE
:1042D00088830091730510E0C7018E569F4F0E949E
:1042E000A40AF801E85BFB4F882319F08081826003
:1042F00002C080818D7F808380917305C82FD0E0BC
:10430000C7018C569F4F0E94A40ACE56DB4F88836C
:1043100080917305C82FD0E0C7018A569F4F0E9435
:10432000A40A90E00E947D1ECC56DB4F888300914A
:10433000730510E0C7018C589F4F0E94A40AF80132
:10434000E85BFB4F882319F08081886002C0808180
:10435000877F808380917305C82FD0E0C7018A587A
:104360009F4F0E94A40AC257DB4F88838091730538
:10437000C82FD0E0C70188589F4F0E94A40A90E040
:104380000E947D1EC057DB4F88830091730510E0AB
:10439000C70186589F4F0E94A40AF801E85BFB4FB3
:1043A000882319F08081806102C080818F7E8083A4
:1043B00080917305C82FD0E0C70184589F4F0E9499
:1043C000A40ACA56DB4F888380917305C82FD0E0BA
:1043D000C70182589F4F0E94A40A90E00E947D1E50
:1043E000C856DB4F88830091730510E0C7018058E1
:1043F0009F4F0E94A40AF801E85BFB4F882319F045
:104400008081806202C080818F7D8083809173056E
:10441000C82FD0E0C7018E579F4F0E94A40AC656EE
:10442000DB4F888380917305C82FD0E0C7018C577C
:104430009F4F0E94A40A90E00E947D1EC456DB4F4D
:1044400088830091730510E0C7018A579F4F0E942F
:10445000A40AF801E85BFB4F882319F0808180648F
:1044600002C080818F7B808380917305C82FD0E04C
:10447000C70188579F4F0E94A40AC256DB4F88830A
:1044800080917305C82FD0E0C70186579F4F0E94C7
:10449000A40A90E00E947D1EC056DB4F88830091E5
:1044A000730510E0C7018C559F4F0E94A40AF801C4
:1044B000E65BFB4F882319F08081816002C0808118
:1044C0008E7F808380917305C82FD0E0C7018A5505
:1044D0009F4F0E94A40ACE55DB4F888380917305BD
:1044E000C82FD0E0C70188559F4F0E94A40A90E0D2
:1044F0000E947D1ECC55DB4F88830091730510E030
:10450000C70180559F4F0E94A40AF801E65BFB4F4C
:10451000882319F08081846002C080818B7F808332
:1045200080917305C82FD0E0C7018E549F4F0E9421
:10453000A40ACA55DB4F888380917305C82FD0E049
:10454000C7018C549F4F0E94A40A90E00E947D1ED8
:10455000C855DB4F88830091730510E0C7018A546A
:104560009F4F0E94A40AF801E65BFB4F882319F0D5
:104570008081886002C08081877F808380917305FD
:10458000C82FD0E0C70188549F4F0E94A40AC65587
:10459000DB4F888380917305C82FD0E0C701865414
:1045A0009F4F0E94A40A90E00E947D1EC455DB4FDD
:1045B00088830091730510E0C701845A9F4F0E94C1
:1045C000A40AF801E65BFB4F882319F08081806420
:1045D00002C080818F7B808380917305C82FD0E0DB
:1045E000C701825A9F4F0E94A40AC255DB4F88839D
:1045F00080917305C82FD0E0C701805A9F4F0E9459
:10460000A40A90E00E947D1EC055DB4F8883009174
:10461000730510E0C7018E539F4F0E94A40AF80152
:10462000E65BFB4F882319F08081806802C080819F
:104630008F77808380917305C82FD0E0C7018C539A
:104640009F4F0E94A40ACE54DB4F8883809173054C
:10465000C82FD0E0C7018A539F4F0E94A40A90E060
:104660000E947D1ECC54DB4F88830091730510E0BF
:10467000C70188539F4F0E94A40AF801E65BFB4FD5
:10468000882319F08081806202C080818F7D8083C1
:1046900080917305C82FD0E0C70186539F4F0E94B9
:1046A000A40ACA54DB4F888380917305C82FD0E0D9
:1046B000C70184539F4F0E94A40A90E00E947D1E70
:1046C000C854DB4F88830091730510E0C7018C52FA
:1046D0009F4F0E94A40AF801E45BFB4F882319F066
:1046E0008081826002C080818D7F8083809173058C
:1046F000C82FD0E0C7018A529F4F0E94A40AC65417
:10470000DB4F888380917305C82FD0E0C7018852A2
:104710009F4F0E94A40A90E00E947D1EC454DB4F6C
:1047200088830091730510E0C70180529F4F0E945B
:10473000A40AF801E45BFB4F882319F080818460B0
:1047400002C080818B7F808380917305C82FD0E069
:10475000C7018E519F4F0E94A40AC254DB4F888329
:1047600080917305C82FD0E0C7018C519F4F0E94E4
:10477000A40A90E00E947D1EC054DB4F8883DF9125
:10478000CF911F910F91FF90EF9008958DE796E0E4
:1047900064E773E00E948232813039F08DE796E061
:1047A00064E773E041E00E94893208958F929F92FE
:1047B000AF92BF92CF92DF92FF920F931F93CF934E
:1047C000DF93F62E4901C82EDD248601000F111F4C
:1047D0005801AC0CBD1CE501CC0FDD1FCC0FDD1F5B
:1047E000C85CD94F18828B819C818430910509F473
:1047F0008EC0853091055CF48230910509F443C088
:10480000833091050CF0BFC09923C4F44FC28730A8
:10481000910509F443C18830910544F48530910530
:1048200009F4DEC0069709F041C207C1883091053E
:1048300009F47AC1099709F039C2E7C18EEF681708
:1048400009F034C282E090E09C838B8380E790E0A3
:10485000C89ED001C99EB00DD89EB00D1124A8539A
:10486000BA4F13961C92139788E390E0C89EF0010C
:10487000C99EF00DD89EF00D1124EE0FFF1FE653D8
:10488000FA4F6083A4C1E5E6E61788F489818F5F5B
:104890008983F501EE0FFF1FEE0FFF1FE65CF94F56
:1048A00080818F5F8083188281E090E02DC080E757
:1048B00090E0C89EF001C99EF00DD89EF00D112425
:1048C000E853FA4F63831D8280818627282F229523
:1048D000207F282730E0522F4427C90163E0880F4A
:1048E000991F6A95E1F748275927818190E0482769
:1048F000592784E0359527958A95E1F74227532774
:104900005183408384E090E09C838B83CFC18CE112
:1049100090E0C89EF001C99EF00DD89EF00D1124C4
:10492000EE0FFF1FEE0FFF1FE453FA4F608380E787
:1049300090E0C89EF001C99EF00DD89EF00D1124A4
:10494000E853FA4F80818627282F2295207F282739
:1049500030E0522F4427C901B3E0880F991FBA9560
:10496000E1F748275927818190E048275927A4E09B
:1049700035952795AA95E1F7422753275183408320
:1049800083E090E0C1CF80E790E0C89EF001C99E2F
:10499000F00DD89EF00D1124E853FA4F6583808105
:1049A0008627282F2295207F282730E0522F442762
:1049B000C90163E0880F991F6A95E1F748275927D5
:1049C000818190E04827592704E0359527950A957D
:1049D000E1F7422753275183408385E090E094CF4D
:1049E00080E790E0C89EF001C99EF00DD89EF00DC2
:1049F0001124E853FA4F668380818627282F229559
:104A0000207F282730E0522F4427C901B3E0880FC8
:104A1000991FBA95E1F748275927818190E04827E7
:104A20005927A4E035952795AA95E1F74227532702
:104A30005183408386E090E067CF80E790E0C89E96
:104A4000F001C99EF00DD89EF00D1124E853FA4FE5
:104A5000678380818627282F2295207F282730E0B2
:104A6000522F4427C90163E0880F991F6A95E1F727
:104A700048275927818190E04827592794E03595A8
:104A800027959A95E1F742275327518340838381E5
:104A9000882309F446C087E090E036CF6D81F801A5
:104AA00083E0EE0FFF1F8A95E1F7E01BF10B3196D3
:104AB00003E0EE0FFF1F0A95E1F7E60FF11DE85343
:104AC000FA4FF0826F5F6D8380E790E0C89EF0013F
:104AD000C99EF00DD89EF00D1124E853FA4F808145
:104AE0008F25282F2295207F282730E0522F44271A
:104AF000C901B3E0880F991FBA95E1F748275927F4
:104B0000818190E048275927A4E035952795AA95FB
:104B1000E1F742275327518340838381681709F0C7
:104B2000C5C088E090E0F0CE80E790E0C89ED0015C
:104B3000C99EB00DD89EB00D1124A853BA4F9C91B8
:104B40001796EC911797F0E0EB5FFC4F8081892777
:104B5000482F4295407F482750E0342F2227CA0132
:104B6000E3E0880F991FEA95E1F728273927119686
:104B70008C91119790E02827392774E05595479537
:104B80007A95E1F72427352711963C932E93862FAB
:104B900090E0307082179307F9F0F501EE0FFF1FD8
:104BA000EE0FFF1FE65CF94F80818F5F80831882D4
:104BB00081E090E09C838B83FEEFFF1609F076C0C6
:104BC00082E090E09C838B8313961C9213978FEF67
:104BD0009FEF8D939C936AC089E090E09C838B83C8
:104BE000F80153E0EE0FFF1F5A95E1F7E01BF10BC0
:104BF000319643E0EE0FFF1F4A95E1F78D81E80FF4
:104C0000F11DE853FA4F608351C0262F30E080E752
:104C100090E0C89EB001C99E700DD89E700D112401
:104C200068537A4FFB01818190E028173907E9F03A
:104C3000F501EE0FFF1FEE0FFF1FE65CF94F8081BD
:104C40008F5F8083188281E090E09C838B83FEEFEE
:104C5000FF1661F582E090E09C838B83EB011B8261
:104C60008FEF9FEF9983888321C081E0888381E063
:104C700090E09C838B83F80123E0EE0FFF1F2A95C1
:104C8000E1F7E01BF10B319693E0EE0FFF1F9A95D1
:104C9000E1F78D81E80FF11DE753FA4FF082DA0159
:104CA000FB0180E701900D928150E1F7D601AA0F38
:104CB000BB1FAC0DBD1DAA0FBB1FAA0FBB1FA85C5D
:104CC000B94F8C91813069F58CE190E0C89EF0017C
:104CD000C99EF00DD89EF00D1124EE0FFF1FEE0FB0
:104CE000FF1FE453FA4F808116968C9316971896FF
:104CF0008D919C911997892B21F41B961C921E92E1
:104D00001A97F601EE0FFF1FEC0DFD1DEE0FFF1FB2
:104D1000EE0FFF1FE85CF94F808591850196918722
:104D20008087F601EE0FFF1FEC0DFD1DEE0FFF1F3C
:104D3000EE0FFF1FDF01A85CB94F16968C911697F6
:104D40008F5FE4018E8318968D919C9119979987B6
:104D50008887E65CF94F80818A871B8610828C9158
:104D6000DF91CF911F910F91FF90DF90CF90BF9077
:104D7000AF909F908F9008954F925F927F928F9205
:104D80009F92AF92BF92CF92DF92EF92FF920F93DA
:104D90001F93DF93CF93CDB7DEB7C854D0400FB683
:104DA000F894DEBF0FBECDBF8FED94E00E942705C3
:104DB00000D000D002EC14E0EDB7FEB712830183FF
:104DC00086E691E0948383830E94C02B3BE5432ECB
:104DD00031E0532EEE24FF24CC24DD240F900F90DD
:104DE0000F900F90702E012F29E0A22EB12CAC0E47
:104DF000BD1E4E010894811C911C82EC94E00E941F
:104E0000742C982F8D3031F08D30DCF1805382304E
:104E1000C0F530C01830A1F59981892F80538230B8
:104E200078F5913311F490E801C090E08A818133E4
:104E300009F4905C8B81813309F4905E8C8181331D
:104E400009F4905F8D81813309F4985F8E818133FD
:104E500009F49C5F8F81813309F49E5F88858133DB
:104E600009F49F5FF501EE0DFF1D90830894E11C8E
:104E7000F11C06C0F401E10FF11D90831F5F01C01A
:104E800010E0F0E4EF16F104C9F48FED94E0B60100
:104E9000A5010E9412040894C11CD11C00D000D0AE
:104EA000EDB7FEB771820283548243820E94C02B09
:104EB000EE24FF240F900F900F900F90FFEFCF166E
:104EC000D10409F00CF499CFC85BDF4F0FB6F8940A
:104ED000DEBF0FBECDBFCF91DF911F910F91FF902D
:104EE000EF90DF90CF90BF90AF909F908F907F908A
:104EF0005F904F900895AF92BF92CF92DF92EF9262
:104F0000FF920F931F93DF93CF93CDB7DEB7CC57AC
:104F1000D0400FB6F894DEBF0FBECDBF8E01035F49
:104F20001F4F5E010894A11CB11CEE24E39445E1DF
:104F3000C42ED12CCC0EDD1EC1C182EC94E00E94A7
:104F4000742CF82E8091B505882311F50E94DD326E
:104F500060527E4480409040D8F40E94DD3269580F
:104F6000734180409040A0F0FAE0FF1619F02DE068
:104F7000F21631F48091B6058F5F8093B60502C0BA
:104F80001092B6058091B605833011F40E94BC26BC
:104F900080E06F2DA80195010E94D623882309F493
:104FA00089C10E94DD320E94BC356093B0057093C8
:104FB000B1058093B2059093B305E092B5058C8955
:104FC0008E3109F4F4C08F3158F4813099F1813079
:104FD000D0F0883109F44EC08D3109F06BC163C146
:104FE0008E3309F407C18F3338F4833209F421C1B9
:104FF0008A3209F05FC118C18A3409F490C0883A36
:1050000009F058C136C1E092B7058A898093B80586
:105010008B898093B905F801808580931A05868570
:105020008093BA05881F8827881F80931B051092DC
:10503000BB0540C1F8016689778980E090E00E9455
:10504000BC3520E030E04AE754E40E942335609309
:105050004305709344058093450590934605F801F8
:10506000808D918D909372058093710586A18093B8
:105070004F0520C1F801608D718D828D938D0E9446
:10508000BE3520E030E04AE754E40E9423350E9418
:105090008B3560936D0570936E0580936F059093CB
:1050A0007005F80160897189828993890E94BE35F3
:1050B00020E836E948E15BE40E9423356093370538
:1050C000709338058093390590933A05F801648907
:1050D0007589868997890E94BE3520E836E948E1BE
:1050E0005BE40E94233560933B0570933C058093FD
:1050F0003D0590933E05F601848D80933F05858D97
:1051000080934205828D938D9093AE058093AD057B
:10511000848995899093410580934005CBC0F60121
:1051200080819181A281B38180935A0590935B0520
:10513000A0935C05B0935D0584819581A681B781BC
:105140008093690590936A05A0936B05B0936C05F5
:10515000F801608D718D882777FD8095982F0E94CA
:10516000BE3560931F0570932005809321059093B1
:105170002205F801828D8093540580899189A28946
:10518000B3898093BC059093BD05A093BE05B093F1
:10519000BF05F60184859585A685B7858093C005F2
:1051A0009093C105A093C205B093C30583C0F801D5
:1051B000608971898289938921EE3EE245E652E455
:1051C0000E94F1360E948B3570930F0560930E0597
:1051D000F801648575858685978521EE3EE245E672
:1051E00052E40E94F1360E948B3570930D05609356
:1051F0000C0560C0F801868D978D90931E058093F5
:105200001D0580A191A190932A0580932905808D89
:10521000918DA28DB38D8093240590932505A09345
:105220002605B093270546C0F801808580932805A0
:1052300041C0F6018485958590937C0580937B051C
:105240008685978590937E0580937D05F801808DF6
:10525000918D9093800580937F05F60182899389D3
:105260009093820580938105F801858D8093910547
:1052700021C0F60180819181A281B3818093840550
:1052800090938505A0938605B093870584819581C9
:10529000A681B7818093100590931105A093120504
:1052A000B093130507C0F8018489958990939C05F4
:1052B00080939B058AE890E00E94443382EC94E05E
:1052C0000E94442C181619060CF437CE8091C405A0
:1052D0009091C5052B853C85820F931F9093C50542
:1052E0008093C4052B818091C6059091C705820FDC
:1052F000911D9093C7058093C605C458DF4F0FB624
:10530000F894DEBF0FBECDBFCF91DF911F910F91FB
:10531000FF90EF90DF90CF90BF90AF90089586E020
:1053200061E00E94C83308950F931F9386E061E007
:105330000E94893302EC14E0C80140E051EE60E0C5
:1053400070E00E94E22B10937F0600937E060E947D
:105350008F298FED94E00E94A6050E94A61B64EFA2
:1053600071E080E090E00E94EB320E94310A1092DE
:10537000730507C00E94921E809173058F5F809312
:105380007305809173058230A8F31092730560ED68
:1053900077E080E090E00E94EB3282EC94E00E94A3
:1053A000C12C1F910F9108952F923F924F925F92BF
:1053B0006F927F928F929F92AF92BF92CF92DF9225
:1053C000EF92FF920F931F93DF93CF9300D000D003
:1053D000CDB7DEB7E090BC05F090BD050091BE05ED
:1053E0001091BF05C801B7012091590630915A06A6
:1053F00040915B0650915C060E945534609308050D
:105400007093090580930A0590930B0590911B05F5
:1054100080915D06981721F081E089278093B4057B
:1054200090935D06A090B405AA2059F580913F05A0
:10543000823008F43BC18091370590913805A091E6
:105440003905B0913A0580935E0690935F06A0936C
:105450006006B093610680913B0590913C05A09158
:105460003D05B0913E058093620690936306A0933C
:105470006406B09365061092660681E08093B405D9
:1054800015C181E0A81609F011C160906606E8E137
:10549000E61580F160916706709168068091690653
:1054A00090916A06A80197010E9455349F7720E0E9
:1054B00030E040E05FE30E94E63618165CF410929C
:1054C0006606E0926706F0926806009369061093FC
:1054D0006A0610C0862D8F5F80936606893151F46D
:1054E000E0925906F0925A0600935B0610935C0610
:1054F000A0924806E0905E06F0905F06009160067C
:1055000010916106C801B7019F7725E33AEF4EE895
:105510005CE30E94F1360E94203569837A838B8395
:105520009C83C801B701209137053091380540911F
:10553000390550913A050E9455341B012C019F7783
:1055400020EC3BE649ED57E40E94F1365B016C012B
:105550006091620670916306809164069091650681
:1055600020913B0530913C0540913D0550913E0511
:105570000E9455343B014C019F7720EC3BE649EDFE
:1055800057E40E94F13629813A814B815C810E9467
:10559000F1367B018C01C601B501A60195010E947F
:1055A000F1365B016C01C801B701A80197010E94A7
:1055B000F1369B01AC01C601B5010E9456340E9430
:1055C00078370E948B356093470570934805809328
:1055D000490590934A0560E070E080E89FE32981E7
:1055E0003A814B815C810E9423359B01AC01C20151
:1055F000B1010E94F13697FA909497F89094A40123
:1056000093010E94C93420EE3EE245E652E40E9436
:10561000F13620E030E044EB52E40E9456340E9420
:105620008B359B01AC0197FF04C028593E4F4F4F6B
:105630005F4FCA01B901645B70408040904097FFA2
:1056400006C0CA01B9016C547F4F8F4F9F4F0E9413
:10565000BE3520911F0530912005409121055091C4
:1056600022050E9455340E948B3597FF04C068596B
:105670007E4F8F4F9F4F0E94BE3520E030E044EBBD
:1056800053E40E94233520E030E040E851E40E94DA
:10569000F1360E9454370E948B35DC01CB0160E16A
:1056A00070E00E944A388F5F80931C050F900F9026
:1056B0000F900F90CF91DF911F910F91FF90EF907E
:1056C000DF90CF90BF90AF909F908F907F906F9022
:1056D0005F904F903F902F9008950E947A0D8FED2C
:1056E00094E00E94D4290E94AB1B0E94AA070E944A
:1056F000C62308950E94DD3220914406309145066C
:10570000409146065091470628583F4F4F4F5F4FF4
:10571000261737074807590760F40E94DD32609367
:1057200044067093450680934606909347060E9470
:105730006D2B0E947B2708956EBD0DB407FEFDCF33
:105740008EB508958DE061E00E9489338BE061E0C1
:105750000E9489338CE060E00E9489338AE061E036
:105760000E9489331CBC80E58CBD8DB58EB5089533
:105770008BE696E00E94A22B08958FEF9FE7089595
:10578000DF93CF93CDB7DEB7FE0139968D819E8131
:1057900061E04F8158859F010E94612ECF91DF917A
:1057A0000895DF93CF93CDB7DEB7FE0139968D8193
:1057B0009E8160E04F8158859F010E94612ECF91AC
:1057C000DF9108950F931F93DC01ED91FC91028806
:1057D000F389E02D20E030E000E010E009951F9112
:1057E0000F9108958F92AF92CF92EF92FF920F9305
:1057F0001F93DF93CF93CDB7DEB7FC0113821282E4
:1058000088EE93E0A0E0B0E084839583A683B7831D
:105810008DE294E09183808355874487378726877C
:10582000118B008BF38AE28AC48AA58A868A70E08B
:10583000CB0123E0880F991F2A95E1F79C01245999
:10584000394F308F278B8C58994F928F818F81E001
:1058500090E002C0880F991F6A95E2F720917C06BC
:10586000282B20937C06CF0140E051EE60E070E0F1
:105870000E94E22BCF91DF911F910F91FF90EF904B
:10588000CF90AF908F900895FC01838D882319F4F9
:105890002FEF3FEF0DC00788F08DE02D2081318183
:1058A00082819381281B390B848195812823392398
:1058B000C9010895FC01838D882319F42FEF3FEF70
:1058C00011C0018CF28DE02D208131818281938184
:1058D000281B390B20953095848195812823392305
:1058E0002F5F3F4FC9010895FC01838D882361F02C
:1058F000A789B08D2D913C91119712968D919C9115
:1059000013972817390721F44FEF5FEFCA01089565
:1059100012968D919C9113971696ED91FC91179785
:10592000E80FF91F408112968D919C911397019673
:1059300014962D913C9115978223932313969C9353
:105940008E93129750E0E2CFFC01838D882351F0B3
:105950000788F08DE02D2081318182819381281785
:10596000390721F42FEF3FEFC90108958281938118
:105970000680F781E02DE80FF91F8081282F30E0A5
:10598000F3CFDC015796ED91FC915897828193817A
:10599000918380835996ED91FC915A9780819181F2
:1059A000938382830895DC015B968C915B978823B7
:1059B000A9F15996ED91FC915A97208131812F5F81
:1059C0003F4F84819581282339235C968C915C9785
:1059D000882329F08281938128173907F9F0828181
:1059E000938128173907D9F3808191810680F78147
:1059F000E02DE80FF91F60835996ED91FC915A97BD
:105A0000318320835296ED91FC9153978081569675
:105A10009C91892B808321E030E002C020E030E0BF
:105A2000C9010895CF93DF93EC011B821A828A810A
:105A30009B81998388831D821C828E819F81009720
:105A400021F00E9475031F821E82DF91CF9108957D
:105A50000F931F938C01DC015296ED91FC915397AB
:105A6000208156968C91569755969C915597892BE7
:105A700080958223808357968D919C9158970E94A0
:105A8000122DF801818D928D0E94122DD8015B9606
:105A90001C921F910F9108950F931F93CF93DF9343
:105AA0008C01FC0113821282828193819183808315
:105AB00041E0A1E0B0E001C04F5FFD01042E02C053
:105AC000EE0FFF1F0A94E2F79B0182E06130780736
:105AD00010F020E032E0E217F30770F3C1E0D0E00D
:105AE00002C0CC0FDD1F4A95E2F72197F80126810D
:105AF00037812115310541F0848195818C179D07EF
:105B000089F0C9010E947503F801D583C483CE01D1
:105B100001960E94CB029C01F8019783868380E066
:105B2000232B09F081E0DF91CF911F910F91089510
:105B3000AF92BF92CF92DF92EF92FF920F931F939B
:105B4000CF93DF937C015A016B01E901DC015B9685
:105B50008C915B978823F1F02115310539F4579624
:105B6000ED91FC915897C481D581219601151105BD
:105B700049F4D7015996ED91FC915A97048115810A
:105B80000F5F1F4FD701ED91FC910088F189E02D47
:105B9000C7010995F7018789908D209711F4C0E816
:105BA000D0E0BE010E944C2D882381F0D701599688
:105BB0008D919C915A970115110511F400E110E0A7
:105BC000B8010E944C2D882309F04DC0D701ED91FA
:105BD000FC910088F189E02DC701099567C0D701C4
:105BE0005096ED91FC915197B0E0AB16B1EEBB062B
:105BF000B0E0CB06B0E0DB0609F454C081E090E0F1
:105C0000D70154960C9002C0880F991F0A94E2F7AE
:105C1000808360E079E08DE390E0A60195010E9429
:105C20007F382150304040405040CA01B90122E045
:105C300030E040E050E00E947F38D7011C96ED91A3
:105C4000FC911D9730831E96ED91FC911F97208348
:105C5000D7015296ED91FC915397808155969C9176
:105C6000892B808323C0D7015996ED91FC915A97D7
:105C70001382128282819381918380835796ED9162
:105C8000FC91589713821282828193819183808341
:105C900081E05B968C931A141B041C041D040CF405
:105CA0009ECFD6CF108220E130E0C7CFDF91CF91D9
:105CB0001F910F91FF90EF90DF90CF90BF90AF902A
:105CC00008952F923F924F925F926F927F928F92A0
:105CD0009F92AF92BF92CF92DF92EF92FF920F937B
:105CE0001F93DF93CF93CDB7DEB764970FB6F894C9
:105CF000DEBF0FBECDBF3C01688B5A8B498B69015B
:105D00001C01AE014F5F5F4F5C8B4B8BE989FA89B9
:105D1000488940FD659140FF6191FA8BE98B6623CC
:105D200009F4D7C3653249F440FD859140FF819164
:105D3000FA8BE98B8532B1F40CC06A3051F4D3018F
:105D4000ED91FC910190F081E02DC1016DE009958C
:105D50006AE0D301ED91FC910190F081E02DC10149
:105D60000995D4CF982F10E0882499241032B0F4EC
:105D70009B3269F09C3228F4903251F0933271F4E6
:105D80000BC09D3239F0903349F4116028C0126085
:105D9000146025C0186023C0106121C017FD2BC0FE
:105DA000892F80538A3078F416FF06C0BAE09B9E94
:105DB000902C1124980E13C0EAE08E9E802C1124A2
:105DC000880E10620CC09E3221F416FD82C310644E
:105DD00006C09C3611F4106802C0983661F4E98957
:105DE000FA89488940FD959140FF9191FA8BE98BA2
:105DF000992309F0BBCF892F8554833020F4812F5C
:105E00008061905E07C0892F8556833008F0E6C117
:105E1000812F8F7E86FD02C076E0972E6FE3F62EEF
:105E2000F822953619F450E4F52A07C0963619F48D
:105E300080E8F82A02C091109A94F7FE0BC09BE309
:105E4000991520F427E05CE3B52E0DC0B92CB3946E
:105E500027E009C0A7E0A91520F447E0942E27E029
:105E600001C0292DBB24F6013496FD87EC87D601AD
:105E70006D917D918D919C91AE014F5F5F4F0B2D88
:105E80000E9495016C010981E02FF0E0FF87EE8709
:105E900000FF05C0FE85F3FD02C01DE209C0F1FE52
:105EA00002C01BE205C0F2FC02C010E001C010E21B
:105EB0008E859F858C709070892B09F444C01123C6
:105EC00011F483E001C084E0881510F088240EC02E
:105ED000881AF3FC0BC0D301ED91FC910190F08185
:105EE000E02DC10160E209958A94A9F7112349F0D8
:105EF000D301ED91FC910190F081E02DC101612F62
:105F00000995BE85B3FF03C000E712E012C004E7A5
:105F100012E00FC0E114F10409F06052D301ED91D9
:105F2000FC910190F081E02DC10109950F5F1F4F99
:105F300005C0EF2CFF24B0E1EB22FF24F8016491AF
:105F4000662341F748C1F7FE13C0BC0CFE85F4FF81
:105F500004C08A81813309F4BA941B141CF0BB2459
:105F6000B3942DC048E04B1550F538E0B32E27C050
:105F7000F6FC25C0892D90E08C159D054CF05CEF5A
:105F8000C5165FEFD50624F080E8F82A01C09A9480
:105F9000992049F0E2E0F0E0EC0FFD1FE90DF11D62
:105FA00080818033A1F3F7FE0AC0B92CB394892D08
:105FB00090E0C816D90614F0992401C09C18F7FC8B
:105FC00003C025E030E009C01C141D041CF021E0D2
:105FD00030E003C096012F5F3F4F112311F02F5F78
:105FE0003F4F992029F0892D90E00196280F391F05
:105FF000882D90E02817390714F0882401C0821AF0
:106000004F2C5524C20189709070892B59F00CC017
:10601000D301ED91FC910190F081E02DC10160E28E
:1060200009958A948820A1F7112349F0D301ED91B5
:10603000FC910190F081E02DC101612F099543FE93
:106040000BC00CC0D301ED91FC910190F081E02DCB
:10605000C10160E309958A948820A1F7F7FE51C039
:106060008601D7FE02C000E010E076010894E11C32
:10607000F11CE01AF10AE1E0F0E0EC0FFD1FEE0E7A
:10608000FF1E26014B185108892D90E0AA24BB243D
:10609000A81AB90AFFEF0F3F1F0749F4D301ED918A
:1060A000FC910190F081E02DC1016EE20995C016CE
:1060B000D10634F0401651061CF4F701608101C08E
:1060C00060E3015010400894E11CF11C0A151B0507
:1060D0004CF0D301ED91FC910190F081E02DC101D4
:1060E0000995D8CF0C151D0541F48A81863320F41B
:1060F000853319F4BE85B4FF61E3D301ED91FC91C2
:1061000065C06A81613309F00F7ED301ED91FC9186
:106110000190F081E02DC10109959920E1F0D301B2
:10612000ED91FC910190F081E02DC1016EE20995A5
:1061300012E0E1E0F0E0EC0FFD1FE10FF11D6081E6
:106140001F5FD301ED91FC910190F081E02DC10121
:1061500009959A9471F7D301ED91FC910190F0812A
:10616000E02D44FC02C065E601C065E4C10109956B
:10617000D7FC05C0C114D10441F404FF06C0D0947B
:10618000C194D108D3946DE201C06BE2D301ED91CB
:10619000FC910190F081E02DC101099560E305C0FB
:1061A0006F5FE6EFFFEFCE0EDF1EFAE0CF16D104F1
:1061B000BCF7D301ED91FC910190F081E02DC1017C
:1061C0000995D301ED91FC916C2D605D0190F081FA
:1061D000E02DC1010995CC84DD8478C1933631F07E
:1061E000933799F0933509F061C023C0F60180819F
:1061F00089835E010894A11CB11C42E050E0C40EEA
:10620000D51E21E0E22EF12C12C0D601AD90BC903B
:1062100016FD03C06FEF7FEF02C0692D70E0E2E072
:10622000F0E0CE0EDF1EC5010E94D8037C011F776F
:1062300013C0D601AD90BC9016FD03C06FEF7FEF89
:1062400002C0692D70E0E2E0F0E0CE0EDF1EC50175
:106250000E94CD037C01106813FF0BC023C0D30143
:10626000ED91FC910190F081E02DC10160E2099572
:106270008A94882D90E0E816F90688F313C0F5019A
:1062800017FD659117FF61915F01D301ED91FC91BD
:106290000190F081E02DC101099581108A94089444
:1062A000E108F108E114F10451F710C1943611F03E
:1062B000993699F517FF0AC0F60120813181428194
:1062C000538184E090E0C80ED91E0CC0D6018D9198
:1062D0009C919C01442737FD4095542FE2E0F0E06B
:1062E000CE0EDF1E9FE6F92EF12257FF09C0509512
:1062F0004095309521953F4F4F4F5F4FF0E8FF2A73
:10630000CA01B901AE014F5F5F4F2AE030E00E9441
:106310006D02E82E4B89E41A41C0953721F41F7EA7
:106320002AE030E01CC0197F9F3661F0903720F4DE
:10633000983509F0CEC00FC0903739F0983709F082
:10634000C8C004C028E030E00AC0106114FD146029
:1063500020E130E004C014FD166020E132E017FFB8
:1063600008C0D6016D917D918D919C91E4E0F0E0A3
:1063700008C0D6018D919C91BC0180E090E0E2E0E4
:10638000F0E0CE0EDF1EAE014F5F5F4F0E946D0248
:10639000E82EFB89EF1A8FE7F82EF122F6FE0BC0EC
:1063A0004EEFF422E91438F4F4FE07C0F2FC05C005
:1063B0005FEEF52202C01E2D01C0192DF4FE0DC0A6
:1063C000FE01EE0DF11D8081803319F489EEF82273
:1063D00008C01F5FF2FE05C003C08F2D867809F04C
:1063E0001F5F0F2DF3FC18C0F0FE13C0181510F03E
:1063F0009E2C0FC09E2C980C911A182D0AC0D30108
:10640000ED91FC910190F081E02DC10160E20995D0
:106410001F5F1815A0F304C0181510F4811A01C0ED
:10642000882404FF17C0D301ED91FC910190F08105
:10643000E02DC10160E3099502FF29C0D301ED9170
:10644000FC910190F081E02D01FD02C068E712C0CF
:1064500068E510C0802F8678D1F001FF02C06BE2A2
:1064600001C060E2F7FC6DE2D301ED91FC91019077
:10647000F081E02DC10109950AC0D301ED91FC9195
:106480000190F081E02DC10160E309959A94E9142F
:10649000A0F3EA94D301ED91FC91A1E0B0E0AC0F40
:1064A000BD1FAE0DB11D0190F081E02DC1016C91B9
:1064B0000995EE2071F70AC0D301ED91FC9101908E
:1064C000F081E02DC10160E209958A948820A1F74E
:1064D0001DCC64960FB6F894DEBF0FBECDBFCF9132
:1064E000DF911F910F91FF90EF90DF90CF90BF90C1
:1064F000AF909F908F907F906F905F904F903F9064
:106500002F900895F999FECF72BD61BDF89A80B5BC
:106510000895F999FECF1FBA72BD61BD40BD0FB697
:10652000F894FA9AF99A0FBE08951F920F920FB637
:106530000F9211242F933F938F939F93AF93BF9309
:106540008091840690918506A0918606B091870679
:10655000309188060196A11DB11D232F2D5F2D3787
:1065600020F02D570196A11DB11D20938806809320
:10657000840690938506A0938606B0938706809143
:10658000800690918106A0918206B09183060196C3
:10659000A11DB11D8093800690938106A093820671
:1065A000B0938306BF91AF919F918F913F912F91AF
:1065B0000F900FBE0F901F9018958FB7F8942091F1
:1065C00084063091850640918606509187068FBFDC
:1065D000B901CA0108959B01AC017FB7F89480917D
:1065E000800690918106A0918206B091830666B5DF
:1065F000A89B05C06F3F19F00196A11DB11D7FBF7B
:10660000BA2FA92F982F8827860F911DA11DB11D84
:1066100062E0880F991FAA1FBB1F6A95D1F7BC01C2
:106620002DC0FFB7F8948091800690918106A091CB
:106630008206B0918306E6B5A89B05C0EF3F19F02E
:106640000196A11DB11DFFBFBA2FA92F982F882732
:106650008E0F911DA11DB11DE2E0880F991FAA1F89
:10666000BB1FEA95D1F7861B970B885E9340C8F253
:10667000215030404040504068517C4F2115310539
:106680004105510571F60895019739F0880F991F5A
:10669000880F991F02970197F1F70895789484B5B0
:1066A000826084BD84B5816084BD85B5826085BD0E
:1066B00085B5816085BDEEE6F0E0808181608083F4
:1066C000E1E8F0E0108280818260808380818160D7
:1066D0008083E0E8F0E0808181608083E1EBF0E09E
:1066E000808184608083E0EBF0E080818160808342
:1066F000EAE7F0E08081846080838081826080832B
:106700008081816080838081806880831092C10055
:106710000895CF93DF93482F50E0CA0186559D4FCF
:10672000FC0134914A565D4FFA018491882369F146
:1067300090E0880F991FFC01E858FD4FA591B49196
:10674000FC01EE57FD4FC591D491662351F42FB74C
:10675000F8948C91932F909589238C938881892329
:106760000BC0623061F42FB7F8948C91932F909501
:1067700089238C938881832B88832FBF06C09FB782
:10678000F8948C91832B8C939FBFDF91CF910895C8
:10679000482F50E0CA0182549D4FFC012491CA0148
:1067A00086559D4FFC0194914A565D4FFA013491F4
:1067B000332309F440C0222351F1233071F02430F7
:1067C00028F42130A1F0223011F514C02630B1F0A8
:1067D0002730C1F02430D9F404C0809180008F7735
:1067E00003C0809180008F7D8093800010C084B5AD
:1067F0008F7702C084B58F7D84BD09C08091B000C1
:106800008F7703C08091B0008F7D8093B000E32F1D
:10681000F0E0EE0FFF1FEE57FD4FA591B4912FB79B
:10682000F894662321F48C919095892302C08C9171
:10683000892B8C932FBF0895CF93DF930E944E3303
:106840000E949429C0E0D0E00E947A2B2097E1F3C7
:106850000E940000F9CFCF92DF92EF92FF920F9348
:106860001F93CF93DF937C016B018A01C0E0D0E0DE
:106870000FC0D6016D916D01D701ED91FC91019092
:10688000F081E02DC7010995C80FD91F01501040B4
:106890000115110571F7CE01DF91CF911F910F9175
:1068A000FF90EF90DF90CF9008955058BB27AA2714
:1068B0000ED041C201D230F006D220F031F49F3F19
:1068C00011F41EF4C0C10EF4E095E7FBB6C1E92F48
:1068D00054D280F3BA17620773078407950718F03C
:1068E00071F49EF56CC20EF4E0950B2EBA2FA02D1C
:1068F0000B01B90190010C01CA01A0011124FF276D
:10690000591B99F0593F50F4503E68F11A16F04067
:10691000A22F232F342F4427585FF3CF4695379566
:106920002795A795F0405395C9F77EF41F16BA0B2B
:10693000620B730B840BBAF09150A1F0FF0FBB1FD9
:10694000661F771F881FC2F70EC0BA0F621F731F22
:10695000841F48F4879577956795B795F7959E3F7F
:1069600008F0B3CF9395880F08F09927EE0F97950D
:1069700087950895A1D158F080E891E009F49EEF41
:10698000A2D128F040E851E059F45EEF09C05BC1A4
:1069900016C2E92FE078F1D168F3092E052AC1F378
:1069A000261737074807590738F00E2E07F8E02555
:1069B00069F0E025E0640AC0EF6307F8009407FA85
:1069C000DB01B9019D01DC01CA01AD01EF934AD0A1
:1069D000B2D10AD05F91552331F02BED3FE049E46D
:1069E00050FD49EC63CF0895DF93DD27B92FBF77C2
:1069F00040E85FE31616170648075B0710F4D92F27
:106A0000E9D19F938F937F936F93BCD2E8E6F0E038
:106A10001DD191D12F913F914F915F91EED1DD2307
:106A200049F09058A2EA2AED3FE049EC5FE3D078C4
:106A30005D274DDFDF917FC1DCD008F481E0089550
:106A40004AD1E39589C10CD076C13DD140F034D113
:106A500030F021F45F3F19F0F0C05111B1C1F3C023
:106A60008CD198F39923C9F35523B1F3951B550B9A
:106A7000BB27AA2762177307840738F09F5F5F4F11
:106A8000220F331F441FAA1FA9F333D00E2E3AF052
:106A9000E0E830D091505040E695001CCAF729D06C
:106AA000FE2F27D0660F771F881FBB1F26173707BB
:106AB0004807AB07B0E809F0BB0B802DBF01FF27EB
:106AC00093585F4F2AF09E3F510568F0B6C078C1D9
:106AD0005F3FECF3983EDCF3869577956795B79525
:106AE000F7959F5FC9F7880F911D9695879597F940
:106AF0000895E1E0660F771F881FBB1F62177307B9
:106B00008407BA0720F0621B730B840BBA0BEE1FCD
:106B100088F7E095089504D06894B11151C10895A3
:106B200034D188F09F5790F0B92F9927B751A0F032
:106B3000D1F0660F771F881F991F1AF0BA95C9F711
:106B400012C0B13081F03BD1B1E0089538C1672F58
:106B5000782F8827B85F39F0B93FCCF386957795C1
:106B60006795B395D9F73EF49095809570956195AA
:106B70007F4F8F4F9F4F0895E89409C097FB3EF4D5
:106B800090958095709561957F4F8F4F9F4F99237A
:106B9000A9F0F92F96E9BB279395F69587957795F8
:106BA0006795B795F111F8CFFAF4BB0F11F460FFB8
:106BB0001BC06F5F7F4F8F4F9F4F16C0882311F010
:106BC00096E911C0772321F09EE8872F762F05C024
:106BD000662371F096E8862F70E060E02AF09A95BF
:106BE000660F771F881FDAF7880F9695879597F9B4
:106BF0000895990F0008550FAA0BE0E8FEEF16164E
:106C00001706E807F907C0F012161306E407F507A0
:106C100098F0621B730B840B950B39F40A2661F014
:106C2000232B242B252B21F408950A2609F4A140B7
:106C3000A6958FEF811D811D089597F99F6780E8C4
:106C400070E060E008959FEF80EC0895DF93CF93AC
:106C50001F930F93FF92EF92DF927B018C01689458
:106C600005C0DA2EEF01C9D0FE01E894A591259167
:106C7000359145915591AEF3EF0129DEFE01970163
:106C8000A801DA9479F7DF90EF90FF900F911F91B0
:106C9000CF91DF9108959F938F937F936F93FF938D
:106CA000EF939B01AC019DD0EF91FF91CFDF2F912E
:106CB0003F914F915F9195C000240A9416161706D4
:106CC00018060906089500240A94121613061406DD
:106CD00005060895B8CF59D0E8F3E894EFEFBB2745
:106CE0003FE048EC5FE76B3D73078407950708F1C9
:106CF000FF279F57B25A6A4D7F40894CF04032F4CB
:106D0000BE556542704F8643FF4F0894EE1F915069
:106D100030F0BB0F661F771F881FFF1FEBCF9EE76A
:106D2000882332F0BB0F661F771F881F9A95C1F723
:106D30009395E09565C1092E0394000C11F4882306
:106D400052F0BB0F40F4BF2B11F460FF04C06F5F23
:106D50007F4F8F4F9F4F0895EF93E0FF06C0A2EA49
:106D60002AED3FE049EC5FEBB2DDE5DF0F900394E5
:106D700001FC9058E5E9F0E08ECF57FD9058440FA4
:106D8000551F59F05F3F71F04795880F97FB991F8A
:106D900061F09F3F79F08795089512161306140647
:106DA000551FF2CF4695F1DF08C0161617061806D4
:106DB000991FF1CF86957105610508940895E894AF
:106DC000BB2766277727CB0197F9089512DF08F4D0
:106DD0008FEF08959B01AC0160E070E080E89FE3D5
:106DE00032CE0BD0A8CF68DF28F06DDF18F09523E6
:106DF00009F023CF28CF1124E3CFBFDFA0F3959F65
:106E0000D1F3950F50E0551F629FF001729FBB2791
:106E1000F00DB11D639FAA27F00DB11DAA1F649F3D
:106E20006627B00DA11D661F829F2227B00DA11DF0
:106E3000621F739FB00DA11D621F839FA00D611D76
:106E4000221F749F3327A00D611D231F849F600D97
:106E5000211D822F762F6A2F11249F5750408AF0D0
:106E6000E1F088234AF0EE0FFF1FBB1F661F771F5C
:106E7000881F91505040A9F79E3F510570F0DDCE1C
:106E80009FCF5F3FECF3983EDCF38695779567954F
:106E9000B795F795E7959F5FC1F7FE2B880F911D7A
:106EA0009695879597F9089570DFE0F09E37D8F0B2
:106EB0009639B8F49E3848F4672F782F8827985F62
:106EC000F9CF86957795679593959539D0F3B62F39
:106ED000B1706B0F711D811D20F4879577956795B3
:106EE000939573C08DC06CCF11F40EF4ACCE88C0F6
:106EF0004CDFD0F39923D9F3CEF39F57550B87FF7F
:106F00008FD056959795B0E020F4660F771F881FB5
:106F1000BB1F1F930F9300249001A0018001F0017B
:106F2000A0E80E0F1F1F0A1E511D601B710B800968
:106F3000B50B48F4600F711F801DB51F0E1B1F0B92
:106F40000A0A510907C02E0F3F1F4A1F0E0F1F1FAD
:106F50000A1E511D660F771F881FBB1FA695F79548
:106F6000E795F8F60617170708065B07211D311D80
:106F7000411D0F911F91B901842F9158880F96954B
:106F8000879508959B01AC012CCFDF93D92FA3DE09
:106F9000E695D7952AED3FE049E45FE3B33A62070F
:106FA000730784079507D7952AF0A2EA49EC906801
:106FB0008EDCC1DEE3EBF0E06EDEDD0F0BF00ADF0E
:106FC000DD0F0BF49058DF910895882371F4772337
:106FD00021F09850872B762F07C0662311F499274C
:106FE0000DC09051862B70E060E02AF09A95660FF4
:106FF000771F881FDAF7880F9695879597F9089578
:107000009F3F49F0915028F4869577956795B795FD
:107010009F5F80389F4F880F9695879597F90895C1
:1070200091505040660F771F881FD2F70895629FD6
:10703000D001739FF001829FE00DF11D649FE00D70
:10704000F11D929FF00D839FF00D749FF00D659FD1
:10705000F00D9927729FB00DE11DF91F639FB00DD0
:10706000E11DF91FBD01CF0111240895AA1BBB1B0F
:1070700051E107C0AA1FBB1FA617B70710F0A61B38
:10708000B70B881F991F5A95A9F780959095BC0159
:10709000CD01089597FB092E07260AD077FD04D06D
:1070A000E5DF06D000201AF4709561957F4F0895B2
:1070B000F6F7909581959F4F0895A1E21A2EAA1B8D
:1070C000BB1BFD010DC0AA1FBB1FEE1FFF1FA21798
:1070D000B307E407F50720F0A21BB30BE40BF50B95
:1070E000661F771F881F991F1A9469F7609570951E
:1070F000809590959B01AC01BD01CF01089597FB50
:10710000092E05260ED057FD04D0D7DF0AD0001C6B
:1071100038F450954095309521953F4F4F4F5F4F34
:107120000895F6F790958095709561957F4F8F4FF4
:107130009F4F0895EE0FFF1F0590F491E02D0994E5
:04714000F894FFCFF1
:10714400256300256325332E306625637C2563255E
:107154006325322E30662563002563256325346953
:1071640025630025632563007374616200616372A3
:107174006F00616C7468006175746F006775696491
:10718400006C6F6974007265746C006369726300EB
:10719400706F7369006C616E64006F666C6F00647D
:1071A4007269660000737072740025632573256329
:1071B4000025342E30662563002531302E36667C5A
:1071C4002531302E36660025632532690025352E9B
:1071D400326625630025346925632563002563250C
:1071E400352E3066256300253269256325303269E2
:1071F40000256325332E3069256300256325342E4D
:10720400306625630025332E306925630020202055
:1072140020202020202020202000204E6F204750B6
:107224005320666978210048696768205653706561
:1072340065642100204F7665725370656564212072
:107244000042617474657279204C6F7721002020AC
:107254004C6F772052737369202000257300253307
:107264002E306625630025352E30662563002563A0
:1072740025342E306625632563002563253369256F
:10728400630025632532692563253032690025357D
:107294002E31662563002563253369256325303245
:1072A400697C256325356925637C25632535692536
:1072B400637C256325356925637C2563253569252C
:1072C400637C25632531302E36667C256325313079
:1072D4002E366600256325352E3266256300256328
:1072E4002563253269256325342E306625637C00A9
:1072F40025632563256325342E30662563004F53AB
:107304004420496E697469616C697A65642C2072E1
:1073140065626F6F740020008D060000010000801C
:10732400BF9DFF0164202020202020202000FFFF9B
:10733400FFFFFF000000000A052B3408040B040EB5
:10734400041104BD2B327C8900EDD968770000005C
:10735400590000000000000000D69FDCA81817AAFE
:1073640090437327F6B968EDF4DED409FEE61C1CDD
:1073740084DDE80B992927D6DF8D210F036418EFEC
:10738400EE1EF0B7828200941500347C00000014D5
:1073940000988F0000000000000000000000E7B724
:1073A4003F3600000000000000AF669ED0380000A9
:1073B40000000000000000000000000000000000C9
:1073C40000000000000000000000000000000000B9
:1073D400000000000000000000000086DBD0BC5468
:1073E40016131586004E44BD7F6F151590010000DD
:1073F4000000000000000000000000000000000089
:107404000000000000000000000000000000000078
:107414000000000000000000000000000000000068
:107424000000000000000000000000000000000058
:107434000000000000000000000000000000CC314B
:10744400AA2C532E00828081808180848081808157
:10745400808380818081808580818081800000009C
:1074640000000000000000000000000000D32C2BEE
:1074740034442C742CA42CC12C5A2CE22B282D9887
:027484002D00D9
:00000001FF
